:100000000C94AD040C94CA040C94CA040C94CA0455
:100010000C94CA040C94CA040C94CA040C94CA0428
:100020000C94CA040C94CA040C94CA040C94CA0418
:100030000C94CA040C94E9050C94CA040C94CA04E8
:100040000C94CA040C94CA040C94CA040C94CA04F8
:100050000C941C080C94CA040C94CA040C94CA0492
:100060000C9495060C94CA040C94CA040C94CA040B
:100070000C94BC080C94EB080C94CA0425732D5303
:10008000595354454D2E4C4F470025732E47505819
:100090000025732D4E4D45412E4C4F470054656D44
:1000A000706572617475726520756E6B6E6F776EB8
:1000B0000D0A0054656D703A20252E32660D0A0037
:1000C00042617420766F6C743A20252E33660D0AD7
:1000D0000054696D653A2025752E253032752E2520
:1000E0003034752025753A253032753A2530327511
:1000F0000D0A0057616974696E6720666F72204748
:1001000050530D0A004653204F6B0D0A00465320F2
:100110006572726F722025750D0A004C4F4F50208A
:100120006572723D25750D0A005245535441525473
:100130000D0A00504F5745524F46460D0A00535482
:1001400041525455500D0A0046696C6520636C6F2E
:100150007365640D0A00736F6674752E2E2E004150
:100160006B7475616C697A61636A61004F70656E6A
:100170002025730D0A002B2C3B3D5B5D002A3A3C89
:100180003E7C223F7F0046415433322020200080B5
:100190009A45418E418F804545454949498E8F900A
:1001A00092924F994F555559999A9B9C9D9E9F416C
:1001B000494F55A5A5A6A7A8A9AAABACADAEAFB0AF
:1001C000B1B2B3B4B5B6B7B8B9BABBBCBDBEBFC0A7
:1001D000C1C2C3C4C5C6C7C8C9CACBCCCDCECFD097
:1001E000D1D2D3D4D5D6D7D8D9DADBDCDDDEDFE087
:1001F000E1E2E3E4E5E6E7E8E9EAEBECEDEEEFF077
:10020000F1F2F3F4F5F6F7F8F9FAFBFCFDFEFF0165
:10021000030507090E10121416181C1E4F56004F26
:100220005600494E46004E614E00414343455054EE
:100230000D0A00546F6F20736D616C6C20706F73CA
:100240006974696F6E206368616E67652052454A04
:100250004543540D0A004E45570D0A004449535476
:10026000414E434520444946462052454A45435461
:100270000D0A004E65772064697374616E63653A98
:100280002025666D0D0A004B414C4D414E205245D4
:100290004A4543540D0A0009093C2F74726B73657B
:1002A000673E0A093C2F74726B3E0A3C2F677078D8
:1002B0003E0A000909093C2F74726B70743E0A00F3
:1002C0000909093C74726B7074206C61743D2225BD
:1002D0002E386622206C6F6E3D22252E3866223E17
:1002E0000A090909093C74696D653E25733C2F7440
:1002F000696D653E0A003C3F786D6C2076657273CF
:10030000696F6E3D22312E302220656E636F646905
:100310006E673D225554462D38223F3E0A3C677099
:100320007820786D6C6E733A7873693D22687474C6
:10033000703A2F2F7777772E77332E6F72672F32A1
:100340003030312F584D4C536368656D612D696EA7
:100350007374616E63652220786D6C6E733D2268E4
:100360007474703A2F2F7777772E746F706F67726F
:10037000616669782E636F6D2F4750582F312F318A
:1003800022207873693A736368656D614C6F6361AD
:1003900074696F6E3D22687474703A2F2F77777787
:1003A0002E746F706F6772616669782E636F6D2F40
:1003B0004750582F312F3120687474703A2F2F779F
:1003C00077772E746F706F6772616669782E636FCE
:1003D0006D2F4750582F312F312F6770782E78733B
:1003E00064222076657273696F6E3D22312E312250
:1003F0002063726561746F723D226B346265223EC8
:100400000A093C74726B3E0A09093C74726B73658D
:10041000673E0A007D1D0100632C001E9601A01E90
:100420005A01001F0806101F0606201F0806301F6D
:100430000806401F0606511F0700591F521F5B1F69
:10044000541F5D1F561F5F1F601F0806701F0E00A0
:10045000BA1FBB1FC81FC91FCA1FCB1FDA1FDB1F54
:10046000F81FF91FEA1FEB1FFA1FFB1F801F08066A
:10047000901F0806A01F0806B01F0400B81FB91F70
:10048000B21FBC1FCC1F0100C31FD01F0206E01FFC
:100490000206E51F0100EC1FF31F0100FC1F4E21A7
:1004A0000100322170211002842101008321D02417
:1004B0001A05302C2F04602C0201672C0601752CC4
:1004C0000201802C6401002D260841FF1A03000060
:1004D00061001A03E0001703F8000703FF000100A2
:1004E00078010001300132010601390110014A0191
:1004F0002E017901060180014D0043028101820134
:1005000082018401840186018701870189018A01B2
:100510008B018B018D018E018F0190019101910161
:1005200093019401F60196019701980198013D020B
:100530009B019C019D0120029F01A001A001A2013D
:10054000A201A401A401A601A701A701A901AA0172
:10055000AB01AC01AC01AE01AF01AF01B101B20121
:10056000B301B301B501B501B701B801B801BA01D2
:10057000BB01BC01BC01BE01F701C001C101C20148
:10058000C301C401C501C401C701C801C701CA0133
:10059000CB01CA01CD011001DD0101008E01DE0198
:1005A0001201F3010300F101F401F401F801280143
:1005B000220212013A020900652C3B023B023D0275
:1005C000662C3F0240024102410246020A015302E8
:1005D000400081018601550289018A0158028F017C
:1005E0005A0290015C025D025E025F0293016102A9
:1005F0006202940164026502660267029701960135
:100600006A02622C6C026D026E029C017002710221
:100610009D01730274029F017602770278027902CB
:100620007A027B027C02642C7E027F02A601810298
:100630008202A9018402850286028702AE01440279
:10064000B101B20145028D028E028F029002910229
:10065000B7017B030300FD03FE03FF03AC030400AB
:100660008603880389038A03B1031103C2030200CE
:10067000A303A303C4030803CC0303008C038E036A
:100680008F03D8031801F2030A00F903F303F403FC
:10069000F503F603F703F703F903FA03FA0330044B
:1006A000200350041007600422018A043601C104AB
:1006B0000E01CF040100C004D004440161052604EA
:1006C0000000C700FC00E900E200E400E000E500F3
:1006D000E700EA00EB00E800EF00EE00EC00C400E9
:1006E000C500C900E600C600F400F600F200FB00F9
:1006F000F900FF00D600DC00A200A300A500A7209F
:100700009201E100ED00F300FA00F100D100AA002F
:10071000BA00BF001023AC00BD00BC00A100AB00BC
:10072000BB0091259225932502252425612562256C
:10073000562555256325512557255D255C255B25C7
:100740001025142534252C251C2500253C255E2547
:100750005F255A25542569256625602550256C2579
:100760006725682564256525592558255225532573
:100770006B256A2518250C25882584258C25902530
:100780008025B103DF009303C003A303C303B500B7
:10079000C403A6039803A903B4031E22C603B5032A
:1007A00029226122B1006522642220232123F7003F
:1007B0004822B0001922B7001A227F20B200A025DB
:1007C000A00020202A2A2A204D454E55202A2A2AD8
:1007D0002000256420736174656C697400656C6524
:1007E000203D20252E31666D00656C65203D203F43
:1007F0003F3F0025332E366625630025322E3666B0
:100800002563003F3F3F20452F57003F3F3F204E8D
:100810002F5300506C696B69207A616D6B6E69654E
:10082000746500426C6164206F74772E20706C696F
:100830006B752100426C6164207A616D6B2E706C67
:10084000696B752100426C6164207A61706973750F
:10085000204641542100426C6164207A61706973C2
:10086000752100426C6164206B61727479210042D1
:1008700072616B206B6172747921005374617274C0
:10088000004261746572696120736C61626121006C
:1008900057796C61637A616E69652E2E2E005572F0
:1008A000756368616D69616E69652E2E2E000000AA
:1008B0009A35A135A835B135D935E635ED35B83697
:1008C00000367A36F4355A6170697320616B747939
:1008D000776E79004B61727461204F4B2100475055
:1008E00053204F4B2100437A656B616D206E612070
:1008F0004750532E2E2E000E1F1F1F1F1F1F1F0E8F
:100900001F111F1F1F1F1F0E1F1111111F1F1F0E51
:100910001F11111111111FB1379A3708090A253417
:10092000752D253032752D253032755425303275B0
:100930003A253032753A253032752E3030302573F5
:10094000000303060104060205000305244750477F
:10095000474100244750524D430011241FBECFEFA2
:10096000D0E1DEBFCDBF11E0A0E0B1E0E8EDF5E8F9
:1009700002C005900D92A630B107D9F72AE0A6E093
:10098000B1E001C01D92AD3BB207E1F70E94ED3B23
:100990000C94C1420C9400001F1D1F1E1F1E1F1F20
:1009A0001E1F1E1FCF93DF93EC012C964AE834D014
:1009B0006627772736E4AEE6B1E0532F537009F08F
:1009C0001197321729F078F56A0F7B1F3395F3CF13
:1009D0004CE022D0E8E9F9E030E0C89531963130BA
:1009E00011F451110A94321720F4600D711D3395E2
:1009F000F4CF402D439510D02150A8F0620F711D07
:100A00008827992748E108D015D04CE305D012D0AB
:100A10002CE302D00FD00BC03A912A912417310554
:100A200040F00F900F906FEF7FEF8FEF9FEFDF9110
:100A3000CF91089551E2AA1B08F4A40FA7959795AA
:100A40008795779567955A95B9F7620F711D811D46
:100A5000911D0895CF93DF93FC0120813181428164
:100A60005381CC27DD2757FD3CC0C6E0D1E06CE3C5
:100A70003CD00882198239D00A821B8268E135D0C5
:100A80000C821D82F9012C5F3F4F67E02ED00C864F
:100A90001D869F01A6E4EEE6F1E0BA2FB37009F0DF
:100AA00031972E173F0720F02E1B3F0BA395F3CF56
:100AB000AA871B862E873F87E8E9F9E0AA27C89511
:100AC0003196A13011F4B1110A942015310520F0AE
:100AD00020193109A395F3CFA887198623952E8372
:100AE0003F83CE01DF91CF910895002470E2220F61
:100AF000331F441F551F001C061610F0061A2395BD
:100B00007A95A9F70895A2E0B0E0E9E8F5E00C9441
:100B10007F3F182F0E949308209145023091460292
:100B2000A9014F5F5F4F5093460240934502285EF4
:100B30003E4FF90110834C32F1E05F0788F0F19BE2
:100B40000FC09E012F5F3F4F68E171E08FEB92E095
:100B50000E94A41B892B21F4109246021092450298
:100B600080914502909146028D3221E0920728F053
:100B7000019790934602809345022296E3E00C94FD
:100B80009B3FF8940E946D080E94992760E080E0E6
:100B90000E9490278FE591E00E94822761E088E023
:100BA0000E94902786E591E00E9482271092B00073
:100BB0001092800014BCE0E0FEE7099588E198E01F
:100BC0000FB6F894A895809360000FBE90936000D4
:100BD000FFCF1F920F920FB60F9211242F933F93C6
:100BE0004F935F936F937F938F939F93AF93BF9335
:100BF000EF93FF93CF93DF9300D0CDB7DEB784E3BD
:100C000095E09A838983E981FA8120813181232BC0
:100C100041F0E981FA81208131812150310931830C
:100C20002083029625E08034920759F780916A0567
:100C300090916B050196803526E49207B8F5909364
:100C40006B0580936A050E940E25379B35C0809105
:100C500068059091690501969093690580936805F0
:100C60008C32914051F4F49A809168059091690515
:100C70000196909369058093680588EE93E09093C0
:100C80003F0580933E050E9470088823D1F00E94A2
:100C900077088033B1F40E947708803291F441E004
:100CA00060E281E00E94F7260E94C10510926B0568
:100CB00010926A05F29AC7CF1092690510926805E2
:100CC000E2CF89B190E08095909524E09595879545
:100CD0002A95E1F78F70379B0AC080619091670574
:100CE000891749F080934F058093670504C08111EF
:100CF000F5CF109267050F900F90DF91CF91FF9184
:100D0000EF91BF91AF919F918F917F916F915F9183
:100D10004F913F912F910F900FBE0F901F901895FC
:100D2000E4E3F5E0838D138E08951F920F920FB6C2
:100D30000F921124FF920F931F932F933F934F9382
:100D40005F936F937F938F939F93AF93BF93EF9333
:100D5000FF93CF93DF9300D000D000D0CDB7DEB7A4
:100D60008091780090917900209165053091660519
:100D7000820F931F9093660580936505209164050B
:100D80002F5F2D83209364052F3008F474C09C01DD
:100D900040E050E029833A834B835C83CA01B90168
:100DA0000E94D040F62E072F182F9E839D81892FF9
:100DB00090E0A0E0B0E089839A83AB83BC83BC0160
:100DC000CD010E94D0409B01AC01F9820A831B83B4
:100DD000AE81AC8369817A818B819C810E9428409D
:100DE0002FED35E34DE453E469837A838B839C8351
:100DF00069817A818B819C810E942840462F572FE0
:100E0000BC0149835A836B837C83109266051092E0
:100E10006505109264059A01AB0120934305309358
:100E200044054093450550934605F09B10C02AE9C0
:100E300039E949E550E469817A818B819C810E947E
:100E400082411816C4F4F0981092630514C026E687
:100E500036E646E450E469817A818B819C810E9468
:100E6000234087FFF1CF809163058F5F80936305F7
:100E7000833008F0F09A0F900F900F900F900F9022
:100E80000F90DF91CF91FF91EF91BF91AF919F9123
:100E90008F917F916F915F914F913F912F911F9112
:100EA0000F91FF900F900FBE0F901F90189583B772
:100EB000817F83BF83B7816083BF889583B78E7F2F
:100EC00083BF0895262F6AE070E00E940E3F211133
:100ED00001C00895179AF89470933705609336050A
:100EE0007894F89480913605909137057894892B01
:100EF000C1F71798F8947093370560933605789486
:100F0000F89480913605909137057894892BC1F734
:100F10002150DDCFA2E0B0E0E0E9F7E00C947F3FA4
:100F2000182FF19B3AC081EE92E00E942E1E892B71
:100F300019F087E0809342058FED98E00E9485319B
:100F4000882319F087E0809342051123B1F0409186
:100F50004502509146024115510579F09E012F5FDF
:100F60003F4F68E171E08FEB92E00E94A41B892B58
:100F700021F410924602109245028FEB92E00E94FB
:100F80002E1E892B19F087E08093420588E491E0BA
:100F90000E947A2F87E00E949537F19840E050E058
:100FA00065E080E00E94E7242296E3E00C949B3FFA
:100FB000E1ECF0E01082599A519A509858981092AA
:100FC0006F0510926E058FE290E09093C5008093BC
:100FD000C40080E9808308951092C1000895209193
:100FE0006E0530916F0581E0232B09F480E00895B0
:100FF0009FB7F89420916E0530916F0580E0232B08
:10100000C9F020916C0530916D05F901E459FA4F52
:1010100084812F5F3F4F317030936D0520936C05B5
:1010200020916E0530916F052150310930936F0585
:1010300020936E059FBF08952F932FB72F933F9353
:101040004F935F938F939F93EF93FF935091C600BD
:101050004FB720916E0530916F05F894E0916C05C3
:10106000F0916D05C9010196E20FF31FF170E4598B
:10107000FA4F5483813052E0950758F080916C0507
:1010800090916D050196917090936D0580936C051C
:10109000C90190936F0580936E054FBFFF91EF914B
:1010A0009F918F915F914F913F912F912FBF2F91E2
:1010B0001895E9ECF0E010825B9A539A52985A988E
:1010C0001092B3071092710781E090E09093CD00E9
:1010D0008093CC0088E9808308951092C900089518
:1010E0009091B30781E0911101C080E008954FB75E
:1010F000F8948091B3078823A1F02091B20730E0E3
:10110000F901EE54F84F82812F5F3F4F2F73332741
:101110002093B2079091B30791509093B3074FBFBC
:10112000089580E0FCCF2FB7F894909171072FBFFE
:101130009034C8F73FB720917107F894E091700799
:1011400091E0920FE20FEF73F0E0E059F84F8283E5
:10115000913448F08091700790E001968F73992741
:1011600080937007922F909371073FBF8091C900C1
:1011700080628093C90008952F932FB72F933F93D8
:101180008F939F93EF93FF939091CE003FB7209161
:10119000B307F894E091B20781E0820FE20FEF739A
:1011A000F0E0EE54F84F9283813448F08091B2071A
:1011B00090E001968F7399278093B207822F8093D6
:1011C000B3073FBFFF91EF919F918F913F912F9177
:1011D0002FBF2F9118951F921FB61F9211242F9386
:1011E0003F938F939F93EF93FF9380917107882391
:1011F000D9F03FB7F8948091710720E0882389F0F7
:101200008091700790E0FC01E059F84F228101962F
:101210008F73992780937007809171078150809315
:1012200071073FBF2093CE0080917107811105C0E7
:101230008091C9008F7D8093C900FF91EF919F91AC
:101240008F913F912F911F901FBE1F901895A4E082
:10125000B0E0EDE2F9E00C94803FFC0120813181A7
:1012600042815381CA01B9012496E2E00C949C3F6B
:10127000A4E0B0E0EEE3F9E00C94803FFC019A01B9
:10128000AB01225031094109510985899689A78905
:10129000B08D0297A109B109281739074A075B07E2
:1012A00000F5A185B2850E94653F69837A838B83AF
:1012B0009C8381A592A5A3A5B4A529813A814B81E0
:1012C0005C81280F391F4A1F5B1F29833A834B8398
:1012D0005C8369817A818B819C812496E2E00C9405
:1012E0009C3F19821A821B821C82F3CF9C01AC01A5
:1012F000455F5F4F80E080FB879587F9F9012F5F9D
:101300003F4F9081890F24173507A9F70895CF9390
:10131000DF93DC01ED91FC911197309759F0CF01EB
:10132000EC0128810196203270F02A33C9F7208120
:10133000203319F08FEF9FEF08C032968E179F076A
:10134000C9F78D939C9380E090E0DF91CF91089551
:101350000F931F93CF93DF93EC018B01892B61F4E3
:1013600089E090E020E030E0F80131832083DF91D4
:10137000CF911F910F910895E881F981309781F302
:101380008081882369F32A813B8185819681281792
:10139000390731F781810E94172480FDE1CF288130
:1013A000398180E090E0E0CF8F929F92AF92BF9220
:1013B000EF92FF920F931F93CF93DF93EC018B81FA
:1013C0008823B9F17E0141E3E40EF11C2DA53EA571
:1013D0004FA558A901E010E0B70189810E94782447
:1013E000892BA1F51B820DA51EA52FA538A9898DD6
:1013F0009A8DAB8DBC8D89A09AA0ABA0BCA0B90181
:10140000A801481959096A097B09481759076A0749
:101410007B0778F46A81623061F4A9019801280F92
:10142000391F4A1F5B1F01E010E0B70189810E944C
:10143000782480E090E0DF91CF911F910F91FF9091
:10144000EF90BF90AF909F908F90089581E090E0D3
:10145000F2CFA0E0B0E0EFE2FAE00C947A3FEC01CA
:101460006A017B018DA59EA5AFA5B8A920E030E05B
:101470008C159D05AE05BF05E9F0CE010E94D4098B
:101480009C01892BB9F401E010E0A7019601BE018F
:101490006F5C7F4F89810E941E249C01892B31F053
:1014A00021E030E0CC24CA94DC2C7601CDA6DEA667
:1014B000EFA6F8AAC901CDB7DEB7E8E00C94963FD5
:1014C000A6E0B0E0E6E6FAE00C947C3F8D839E83D4
:1014D000AD81BE8113961C928FEF9FEFDC01ED81F1
:1014E000FE8185A796A7A7A7B0ABCF010E94290AC6
:1014F0008C01892B09F091C0ED81FE81E15DFD4FEA
:10150000E080F180AD81BE81D1968C918B3E21F03F
:10151000885E823008F07AC0B5E5EB16BAEAFB06C1
:1015200081F0ED81FE8184AD95AD8115924031F45D
:10153000AD81BE81DE968C91811128C003E010E060
:101540006EC048E050E066E871E08D819E818D5765
:101550009F4F0E947242892B09F461C0ED81FE8188
:1015600084AD95AD8115924071F4AD81BE81DE965A
:101570008C91882341F090E09C0121503109822315
:101580009323892B59F002E010E049C090E09C01C0
:101590002150310982239323892B81F6ED81FE812D
:1015A000FF9680819181892B89F1ED81FE81EF5B2E
:1015B000FF4F80818150990B029740F5ED81FE81AC
:1015C000EE5BFF4F80819181892B01F1ED81FE81DE
:1015D000EC5BFF4F808191818038910578F48D819B
:1015E0009E818F5A9F4F0E94270969837A838B833C
:1015F0009C83611571058140910540F0ED81FE816C
:10160000E95BFF4F80819181892B49F4F5E5EF1665
:10161000FAEAFF0609F4B7CF91CF04E010E0C80161
:101620002696E6E00C94983FA6E0B0E0EAE1FBE005
:101630000C94723F8D839E836A017B0128013901DE
:1016400032E0C316D104E104F10408F4E5C0ED81F1
:10165000FE8185899689A789B08DC816D906EA06C4
:10166000FB0608F0D9C08081823009F478C083304D
:1016700009F495C0813009F0CFC08A01169507950D
:10168000040F151FC801892F9927869541A152A1E2
:1016900063A174A1480F591F611D711DCF010E94E4
:1016A000290A9C01892B09F04FC08D809E80F1E3AF
:1016B0008F0E911C58013FEFA31AB30AF801F17085
:1016C000E80DF91D81E0C822DD24EE24FF24842DDD
:1016D000C114D104E104F10439F020812F7030E10C
:1016E000439EC0011124822B808381E0ED81FE8125
:1016F000838341A152A163A174A1C501892F9927B8
:101700008695480F591F611D711DCF010E94290A3E
:101710009C01892BC9F4F501F170E80DF91DC11484
:10172000D104E104F104A9F0D301C20154E0B6955B
:10173000A795979587955A95D1F7808381E0ED819C
:10174000FE81838320E030E0C9012696E0E10C941D
:101750008E3F8081807F952D9F70892BEECF7727DC
:101760006F2D5E2D4D2DED81FE8181A192A1A3A152
:10177000B4A1480F591F6A1F7B1FCF010E94290A7D
:101780009C01892B09F7CC0CDD1CF601EE7FF17072
:101790008D819E81E80FF91F12AB01ABCFCFED8198
:1017A000FE8181A192A1A3A1B4A1B701A60127E066
:1017B00076956795579547952A95D1F7480F591F04
:1017C0006A1F7B1FCF010E94290A9C01892B09F007
:1017D000BBCFCC0CDD1CCC0CDD1CFCEFCF22F1E030
:1017E000DF220D811E810F5C1F4F0C0D1D1DC801D6
:1017F0000E9427093FE07322DC01CB01882799274B
:10180000AA27B07F84299529A629B729F8018083C2
:101810009183A283B38392CF22E030E095CFA8E2F8
:10182000B0E0E5E1FCE00C94723F5B01F42EDB01DB
:101830001D921C920E9487096C018BE090E0D7FCFE
:101840001FC0F601EE0FFF1FEA58F74F008111810C
:101850008CE090E00115110599F0F50111830083EA
:10186000E894F0F8D8018C91882399F011968C9126
:101870000E94172480FD0DC0F11006C080E090E0AA
:10188000A896E0E10C948E3F82FFF8CF8AE090E0CA
:10189000F7CFF8011082C1828C2D0E944D2380FD6C
:1018A00050C2FF2011F082FDF1CF40E050E0BA01BC
:1018B000C8010E94600A8230910509F009C26801DE
:1018C000F9E0CF1AFEEFDF0A9E012F5F3F4F79014B
:1018D000480139EC831A3DEF930A5701C6010E9473
:1018E0002709698B7A8B8B8B9C8BD5016D937D93AC
:1018F0008D939D935D01B0E1CB0ED11CC814D9042A
:1019000069F76701E0E1CE0ED11CD7014D915D91E1
:101910006D917D917D0123E030E041155105610518
:10192000710509F4CBC1C8010E94600A9C010297AD
:1019300008F0C4C1D8019D962D913D914D915C91C7
:10194000D097298F3A8F4B8F5C8FDC968D919C912D
:101950008115924009F0C2C1F801E95BFF4F808117
:1019600091819C0140E050E0298B3A8B4B8B5C8B42
:10197000892B49F4C8018B5A9F4F0E942709698B14
:101980007A8B8B8B9C8B89899A89AB89BC89F8016E
:10199000818F928FA38FB48FEF5BFF4FA080D80110
:1019A0001296AC9212978FEF8A0D823008F096C192
:1019B000DE96BC90DE978B2D90E01A969C938E93CA
:1019C0001997009709F48AC19C012150310982239B
:1019D0009323892B09F082C1319680809180F80190
:1019E00090868782C4018F709927892B09F076C170
:1019F000EC5BFF4F808191816C01E12CF12C892BF4
:101A000039F4C8018F5A9F4F0E9427096B017C014E
:101A1000F801FF960190F081E02D309709F45EC146
:101A2000AA2DB0E029893A894B895C890E94653FDB
:101A30006DA37EA38FA398A79F0140E050E02D8F58
:101A40003E8F4F8F58A3C401F4E096958795FA9581
:101A5000E1F7280F391F411D511DDA01C9012DA1E0
:101A60003EA14FA158A5280F391F4A1F5B1F2D8B80
:101A70003E8B4F8B588FC216D306E406F50608F44A
:101A80002DC1D701C601821B930BA40BB50B89A3F3
:101A90009AA3ABA3BCA3CB2CD12CE12CF12CBC0181
:101AA000CD01A70196010E94363F89A19AA1ABA161
:101AB000BCA18C159D05AE05BF0508F40FC1263FDE
:101AC0009FEF390749079FE0590708F007C173E006
:101AD000A72EB12C263FAFEF3A074105510560F420
:101AE000AA24A394B12C263FBFE03B074105510532
:101AF00018F062E0A62EB12C29013A01E2E04E0E68
:101B0000511C611C711CD80155964D925D926D92CD
:101B10007C925897298D3A8D4B8D5C8D5D962D93D7
:101B20003D934D935C939097CD8CDE8CEF8CF8A019
:101B3000C20ED31EE41EF51EF801C1A2D2A2E3A27A
:101B4000F4A2DA01C9012D893E894F89588D820F8F
:101B5000931FA41FB51F81A792A7A3A7B4A7F3E063
:101B6000AF16B10409F0BDC0F801E55AFF4F8081FE
:101B7000918188299929892B09F0B0C0C801835A1D
:101B80009F4F0E9427096B017C01D301C20142E0F3
:101B9000880F991FAA1FBB1F4A95D1F7F801C5A24C
:101BA000D6A2E7A2F0A62C013D01FFEF4F0EF1E017
:101BB0005F1E611C711C89E076946794579447946A
:101BC0008A95D1F729893A894B895C89241535058D
:101BD0004605570508F482C08FEF9FEFDC01F8013E
:101BE000818B928BA38BB48B85879687A787B08BCD
:101BF00080E88483F3E0AF16B10409F049C0F8012E
:101C0000EF59FF4F80819181019709F041C0498DC3
:101C10005A8D6B8D7C8D4F5F5F4F6F4F7F4FC8012B
:101C20000E94290A892BA1F5D80114961C92F8016B
:101C3000E15DFD4F8081918185359A4A49F5C80162
:101C4000C1960E942709623572458146914401F58B
:101C5000C8018B5E9D4F0E942709623772478144FD
:101C60009146B1F4C801875E9D4F0E942709D801B3
:101C700051966D937D938D939C935497C801835E89
:101C80009D4F0E942709F801658776878787908B8B
:101C9000D801AC9280917408909175080196909348
:101CA00075088093740816969C938E93159784EF0D
:101CB00097E01C969C938E931B97E0CDCE14DF0487
:101CC00009F023CE2430310549F481E090E0D8CDED
:101CD00084309105D1F3029708F42CCE8DE090E08A
:101CE000CFCD81149104D1F32DA13EA14FA158A5D0
:101CF000C20ED31EE41EF51E32E0A316B10439F461
:101D0000D301C201880F991FAA1FBB1F47CFA3E0B1
:101D1000B0E0A30192010E94653F6D8B7E8B8F8B9B
:101D2000988FDC01CB01B695A7959795879541E0F3
:101D30004422552466247724840D951DA61DB71DC5
:101D40002DCF83E090E09CCD0F931F93282FFB01B4
:101D5000628D738D80E090E0233059F404891589F9
:101D600020E030E0980111270027602B712B822B97
:101D7000932B1F910F910895A4E0B0E0E2ECFEE0F8
:101D80000C94783F8C016A017B0182E0C816D10473
:101D9000E104F10408F4A7C0F80185899689A789B0
:101DA000B08DC816D906EA06FB0608F09CC08081F3
:101DB000823009F456C0833009F46FC0813009F0D5
:101DC00092C0CA0196958795840F951F9A8389833F
:101DD000892F9927869541A152A163A174A1480F2B
:101DE000591F611D711DC8010E94290A892B39F0F4
:101DF0006FEF7FEFCB012496EAE00C94943FA9802B
:101E0000BA809FEFA91AB90AE981FA81F170E00F4F
:101E1000F11FF1A9F983C501892F99278695F8014A
:101E200041A152A163A174A1480F591F611D711DE9
:101E3000C8010E94290A892BD9F6F501F170E00F3B
:101E4000F11F81A9F981782F6F2FC0FE08C054E0DF
:101E5000769567955A95E1F780E090E0CCCF7F705A
:101E6000FBCF77276F2D5E2D4D2D81A192A1A3A1D0
:101E7000B4A1480F591F6A1F7B1FC8010E94290A7D
:101E8000892B09F0B5CFCC0CDD1CF601EE7FF1708B
:101E9000E00FF11F61A972A9DFCF81A192A1A3A1D7
:101EA000B4A1B701A60127E07695679557954795A8
:101EB0002A95D1F7480F591F6A1F7B1FC8010E943E
:101EC000290A892B09F094CF0F5C1F4FCC0CDD1C25
:101ED000CC0CDD1CC6018C7F9170800F911F0E947D
:101EE00027099F7088CF61E070E080E090E083CFA9
:101EF000A0E0B0E0EEE7FFE00C94723F8C014A01F5
:101F00005B01FC01C081D18181149104A104B10461
:101F100009F068C04D845E846F84788889899A89C5
:101F2000AB89BC894114510461047104B9F04D8935
:101F30005E896F89788D441655066606770670F4BB
:101F4000892B8A2B8B2B91F4C12CD12C7601C701C4
:101F5000B601CDB7DEB7E0E10C948E3F892B8A2B1A
:101F60008B2B91F3412C512C32014394730162016C
:101F70008FEFC81AD80AE80AF80A8D899E89AF89B6
:101F8000B88DC816D906EA06FB0658F0E1E04E16F1
:101F9000510461047104C1F292E0C92ED12CE12CEC
:101FA000F12CB701A601F801808191810E94BC0E3D
:101FB000462F572FBC01411551056105710509F4E4
:101FC00084C04130510561057105C9F04F3F5F4F35
:101FD0006F4F7F4F09F4B0C0C414D504E604F70472
:101FE00039F6B2CFB501A401CE010E94BC0E6B013F
:101FF0007C01F2E0CF16D104E104F10428F4C12CF5
:10200000D12C7601C394A3CF2FEFC216D206E206DD
:10201000F20609F491C08D899E89AF89B88DC816E2
:10202000D906EA06FB0608F492CF49895A896B89DA
:102030007C89452B462B472B09F486CF750164011B
:10204000EFEFCE1ADE0AEE0AFE0AC816D906EA0635
:10205000FB0628F022E0C22ED12CE12CF12CB70196
:10206000A601F801808191810E94BC0E462F572F56
:10207000BC01413051056105710509F24F3FFFEF89
:102080005F076F077F0709F457C0452B462B472B87
:10209000B9F04D845E846F84788822E04216510442
:1020A0006104710450F08D899E89AF89B88D4816FE
:1020B00059066A067B0608F459CF2401350156CF2C
:1020C000C114D104E104F104C1F30FEF1FEF980133
:1020D000B701A601CE010E94140B9C01892B41F58A
:1020E00081149104A104B104C9F4CD86DE86EF8683
:1020F000F88A89899A89AB89BC894D895E896F89FB
:10210000788D4250510961097109481759076A07CA
:102110007B07B8F48C8181608C8319CF970186018D
:10212000B501A401CE010E94140B9C01892BE9F298
:102130002130310509F063CFCC24CA94DC2C760120
:1021400006CF0197A109B109898B9A8BAB8BBC8B08
:10215000E1CFA6E0B0E0EFEAF0E10C94703F5C0163
:102160004B01DC010D90BC91A02DBE83AD83FC0121
:102170004684578460887188F0E24F0E511C611CC0
:10218000711C4114510420E26206710438F0DC0134
:1021900056961D921D921D921C925997F5018689A3
:1021A0009789A08DB18D0097A105B105A9F1B30163
:1021B000A201517066277727452B462B472B09F044
:1021C000D9C00196A11DB11D868B978BA08FB18FB1
:1021D0004289538964897589AD81BE814115510554
:1021E00061057105F9F417968D919C91A0E0B0E01E
:1021F000B301A20135E076956795579547953A95D5
:10220000D1F7481759076A077B0708F4B3C0F501EF
:10221000168A178A108E118E84E090E02696E2E1ED
:102220000C948C3F19968D919C910197A0E0B0E0A1
:102230007301620129E0F694E794D794C7942A9534
:10224000D1F78C219D21AE21BF21892B8A2B8B2B8D
:1022500009F090C08D819E810E94BC0E6B017C01B3
:10226000B2E0CB16D104E104F10418F482E090E06E
:10227000D5CFEFEFCE16DE06EE06FE0619F481E0AE
:1022800090E0CCCFED81FE8185899689A789B08DBC
:10229000C816D906EA06FB0608F45AC08114910450
:1022A00009F4B5CFD50152964D915D916D917C9118
:1022B0005597C5010E94780F6B017C0187E090E083
:1022C000C114D104E104F10409F4A8CFB1E0CB16A4
:1022D000D104E104F10451F2EFEFCE16DE06EE0672
:1022E000FE0669F28D819E810E94D4094C01892BE2
:1022F00031F6B701A6018D819E810E94380969835C
:102300007A838B839C8389819A81AB81BC81ED81A7
:10231000FE8185A796A7A7A7B0AB1F01F1E32F0EFB
:10232000311C80E092E0D101FC011D923197E9F768
:10233000AD81BE8119968D919C918816990680F188
:10234000ED81FE81818592858816990609F097CFE7
:10235000F501C28AD38AE48AF58AB701A6018D8184
:102360009E810E943809D50156966D937D938D9379
:102370009C935997F50146865786608A718A2D810C
:102380003E812F5C3F4F3A83298331E0532289817C
:102390009A81840D951D938F828F80E090E03ECFCF
:1023A00001E010E029813A814B815C81280D391DC3
:1023B000411D511DB101AD81BE8111968C910E94CC
:1023C0007824892B09F0BCCFFFEF8F1A9F0AB0CF7A
:1023D000A0E0B0E0EEEEF1E10C94723F8C016A01F6
:1023E0007B01FC01C081D181C114D104F0E2EF0670
:1023F000F10438F082E090E0CDB7DEB7E0E10C9474
:102400008E3FD701C6018F719927AA27BB27892B39
:102410008A2B8B2B79F7F801C686D786E08AF18A5A
:1024200086809780A084B18481149104A104B104B2
:1024300009F04DC08881833048F08DA19EA1AFA1E5
:10244000B8A50097A105B10509F043C08F81988513
:10245000A0E0B0E0B701A601E5E076956795579555
:102460004795EA95D1F7481759076A077B0710F691
:102470004DA15EA16FA178A5F801468B578B608FA7
:10248000718F828A938AA48AB58A411551056105A4
:10249000710509F4AFCFD701C60129E0B695A7951C
:1024A000979587952A95D1F7840F951FA61FB71F7B
:1024B000868B978BA08FB18FE196F1E0DF22CC0D58
:1024C000DD1DF801D38FC28F80E090E095CFD5015C
:1024D000C40149845A84612C712C39E0440C551C88
:1024E000661C771C3A95D1F74C015D01B501A4013A
:1024F000C414D504E604F70438F4CE010E94380968
:10250000462F572FBC01B8CFF801808191810E94DE
:10251000BC0E4B015C01FFEF8F169F06AF06BF0696
:10252000B1F082E088169104A104B10408F462CFEE
:102530008D899E89AF89B88D88169906AA06BB0633
:1025400008F058CFC418D508E608F708CFCF81E0C7
:1025500090E052CFAEE0B0E0E0EBF2E10C94703FDF
:102560008D879E87AD85BE850D90BC91A02DBA87C5
:10257000A98740E050E0BA018D859E850E94E81150
:102580008C01892B09F0DDC08FEF9FEFDC01ED8519
:10259000FE8580A791A7A2A7B3A722242A94DD24B1
:1025A000DA947C96FC87EB87AD85BE8556964D9177
:1025B0005D916D917C91599789859A850E94290A30
:1025C0008C01892B09F0BDC0ED85FE85E28CF38C72
:1025D000D7013C90332009F4E8C01B969C91892FC9
:1025E0008F738483B5EE3B1621F093FF0FC08F30BD
:1025F00081F02FEFED85FE8520A73FEF31A74FEF4C
:1026000042A75FEF53A7DD24DA9491C08F3009F021
:10261000A5C0AD85BE8597968C91979786FD87C09E
:1026200036FE94C0F7012584E89436F81E968D9105
:102630009D910D90BC91A02DED85FE8580A791A761
:10264000A2A7B3A7D7011D968C911D978211DBCF4E
:102650005A968D919C915B97892BA9F6E985FA850D
:10266000838494848C918F738150990B2DE0289FE3
:102670008001299F100D11242FE0C22E22E0D22EBE
:1026800081E090E0F60125916F01F701E20FF11D65
:10269000A080B180009709F45CC00034110508F0F7
:1026A000B2CF950140E050E029833A834B835C83AD
:1026B000CA01B9010E9423352B013C01A8014F5FDB
:1026C0005F4F5A834983000F111FF401E00FF11F80
:1026D000808191819C0140E050E0CA01B9010E94D3
:1026E00023356D837E838F83988746165706680649
:1026F000790609F088CFC50109811A814CE1C41619
:1027000042E0D40609F0BECFD7012C9126FF0CC0C1
:10271000892B51F0000F111FF401E00FF11F808190
:102720009181892B09F06FCFDD24DA94D30C60E01E
:1027300070E08D859E850E94A9108C01892B09F47B
:1027400033CFC8012E96E2E10C948C3FD3105BCFBF
:1027500079CF3FEFA316B30689F255CFD11005C04C
:10276000C7010E947609821561F3ED85FE8587A178
:1027700080FD09C04BE050E06B857C85C7010E945D
:102780009C42892BF1F2EFEFAD85BE859896EC93D4
:102790009897FFEF9996FC9399972FEF9A962C9321
:1027A0009A973FEF9B963C932ECF04E010E0C9CF61
:1027B000ABE0B0E0EEEDF3E10C94703F8C01DC0196
:1027C0000D90BC91A02DBB83AA83FB015F01819179
:1027D0008F32E1F38C35D1F3F8011682178210861F
:1027E0001186D5018C91803208F44BC07C96F98714
:1027F000E8872A813B812F5C3F4F3B872A87D8019E
:10280000ED91FC914384548442015D824C82E12C21
:10281000F12CF50191915F01292F30E0992309F402
:1028200049C165EB71E0C9010E940C356C0100974C
:1028300009F43DC18032910508F43CC18F32910505
:1028400009F43BC18C35910509F437C180E8C816FD
:10285000D10440F4B6018DE791E00E948A42892BB1
:1028600009F025C19FE3E916F10409F420C1AFEF97
:10287000EA1AFA0AEC81FD81C192D192FD83EC83C0
:10288000C8CF80E887A340E050E0BA01C8010E94A9
:10289000E8119C01C9012B96E2E10C948C3FFC01EC
:1028A0003297E40DF51D208131812032310521F070
:1028B0002E32310509F019C1B1E0EB1AF1080EC151
:1028C000C814D90450F46E147F0409F054C0FBE01E
:1028D0008F16910409F045C004C0EBE08E169104F8
:1028E000B1F5D8015C968C915C97853E19F485E032
:1028F0005C968C93B32DB3603B2E822D8C708C3004
:1029000021F0822D8370833011F4689431F831FC0A
:1029100008C020FE02C0689434F822FE02C0689409
:1029200033F8D80197963C92C8010E94AA129C01E4
:10293000F80187A12115310509F4A2C02430310521
:1029400009F0A8CF82FDA6CF25E030E0A3CF6E141A
:102950007F0439F0B32DB3603B2EE614F70408F47E
:1029600081C0220C220C37019BE0892E912C28E09B
:10297000C22ED12C17C1EC81FD81E038F10508F49D
:1029800057C0F32DF260F983AC81BD81CD01A0E089
:10299000B0E08C839D83AE83BF8345EB51E0BC01E7
:1029A000CD010E94DD348C839D8387FF1FC0EC81A5
:1029B000FD81EF77FF27E157FE4F2491822F90E0B2
:1029C0009D838C83AC81BD81AB2B41F06C817D817B
:1029D00086E791E00E948A42892B61F1B981B36058
:1029E000B983EFE5F0E0FD83EC8318C0AC81BD81D5
:1029F000AF3FB10539F330F3C4010197C816D906CA
:102A000028F0B32DB3603B2E6401CCC0F801EC0D6F
:102A1000FD1D2D81248FC60101966C01F801EC0D7E
:102A2000FD1D3C81348FC60101966C013980BAC00E
:102A30003982CCCF8C819D81815491094A9718F4B9
:102A4000689421F8EBCF8C819D81815691094A973A
:102A500028F7689420F82C813D81205231093D836C
:102A60002C83DCCFF801848D853E11F425E0248F82
:102A700038E08316910409F040CF220C220C3DCFA0
:102A800082FD08CF848184FF5FCF66857785717072
:102A9000EA85FB856E0F7F1FAA81BB818C910E9406
:102AA000A40EF8016683778380879187A8CE26E0FD
:102AB00030E0F0CE84E0382E11C095015901D901E3
:102AC0008C912F5F3F4F8F32C9F38C35B9F391E072
:102AD000803208F090E0392E330C330CC701880F98
:102AE000991FE114F10409F0DACE840D951DFC0163
:102AF00011821082E114F104D1F220E030E0D4011F
:102B00008D919D914D013D832C832F5F3F4F8032EE
:102B10009105A9F3EC81FD81EF2B11F48E9719F447
:102B2000F32DF3603F2EF701EE0FFF1F3297E40DF8
:102B3000F51D808191818E9731F021E0E21AF10834
:102B4000E114F10481F74BE050E060E270E0888529
:102B500099850E94B24248E0842E912CC12CD12C40
:102B6000212C6C807D803FEF631A730A8C819D81DC
:102B7000880F991F840D951DDC010D90BC91A02D2F
:102B8000BD83AC83109709F46DCFA032B10539F045
:102B90009E9709F095CE6E147F0409F498CEB32D5C
:102BA000B3603B2E7D826C82DCCFA6E0B0E0EBED23
:102BB000F5E10C947F3F9C838B837E836D83142F80
:102BC0007A836983CE0101960E9487099C0197FD53
:102BD00024C0220F331FF901EA58F74F0190F0810A
:102BE000E02D309709F01082EB81FC81309709F0DD
:102BF00010822A58374FD901ED93FC9380E01123BE
:102C000069F040E0BE016D5F7F4FCE0105960E94E6
:102C10000F0C2696E3E00C949B3F8BE090E0F9CFFD
:102C2000A1E5B0E0E6E1F6E10C94703F26968FAFA7
:102C3000269727969FAF279725967FAF6EAF25974C
:102C4000F42E27960EAD1FAD2797012B09F436C33E
:102C5000142F1F732A961FAF2A97412FBE016F5B57
:102C60007F4FCE018D5B9F4F0E940F0C2B968FAF35
:102C70002B972C969FAF2C972C962EAD3FAD2C9773
:102C80002C960EAD1FAD2C97232BC9F423968EAD39
:102C90009FAD239729969FAF8EAF29979A838983FB
:102CA00025966EAD7FAD2597CE0101960E94D81373
:102CB0008C01892B79F08F2D8C7181111AC0279688
:102CC000EEADFFAD2797118210822C961FAF0EAF8D
:102CD0002C97E2C288A587FD57C18D819F2D9C71DD
:102CE000911155C184FDE7C2F1FE9BC180FDAAC0D0
:102CF00098C10430110519F769807A8088A5982F4A
:102D0000907A911141C1D3011B96ED91FC91C12C98
:102D1000D12C21913191232B09F097C09CE0FE0129
:102D20007D96DE019D9601900D929A95E1F780FFC8
:102D3000BFC080E488A7812C912C540183948E011C
:102D40000B5D1F4F62961FAF0EAF62971401D30148
:102D50001B962C911B971C969C918BE0FE01BD96B7
:102D6000DE015D9601900D928A95E1F7E22FF92F31
:102D7000B501A401B6E08B16910408F08CC0E9E31C
:102D8000F0E0EC0FFD1F389627E030E0522D5F7029
:102D900040E3450FC10164E0369427946A95E1F75A
:102DA0004A3310F047E3450F215031094293211572
:102DB000310511F0409750F7E9E3F0E0EC0FFD1F0B
:102DC000E20FF31F1EE71083FE017D9680E090E086
:102DD0008217930739F06191AC014F5F5F4F60320A
:102DE00009F05FC0FC017C9681E090E08C0F9D1F94
:102DF000E80FF91F80E22830310548F4A9E3B0E07C
:102E0000AC0FBD1FA20FB31F8C912F5F3F4F81935B
:102E10006296EEACFFAC6297EE16FF0659F7CE0154
:102E200001960E94AA128C010097E9F50FEF801A13
:102E3000900AA00AB00A14E681169104A104B10414
:102E400009F084CF07E010E03ACFBFEFCB1ADB0ADE
:102E500060CF20E130E01A012B01220C331C441C0E
:102E6000551CAC014170552782017101E40EF51E1D
:102E7000011D111DB801A7019695879500FF06C099
:102E800001E2402700E1502701E06027215031098D
:102E90002115310501F7819191910097D1F61A0121
:102EA0006ECFCA0195CF049709F009CF88AD88A7E6
:102EB00088AD81FF3EC0C6010C966DE070E00E94B7
:102EC0000E3F6B012FEFC21AD20AA980BA8040E0F0
:102ED00050E0BA01CE0101960E94E8118C01892BC5
:102EE00019F54F89588D698D7A8DC5010E94290A7F
:102EF0007C01009709F0F1C2EB8DFC8D8081853E4D
:102F000011F0811108C078013FEFE31AF30ACE14E3
:102F1000DF0409F4D9C161E070E0CE0101960E949E
:102F2000A9108C01892B49F00430110509F48ACFCE
:102F3000C6CECC24C394D12CC8CF8701D2CFB9013F
:102F40006F5F7F4F220F331FD201A20FB31F0D916E
:102F50001C9162962EAD3FAD6297820F931FDC01EC
:102F60000D931C930115110561F42416350609F41F
:102F70001EC2FA018491A5014E5F5F4F90E09B0154
:102F8000FBC15A019B0104C206E010E098CE81719A
:102F9000811158CFF2FE50C208E010E090CEF1014E
:102FA00085899689A789B08D481659066A067B06D9
:102FB00008F090C2730162012D96CFAE2D972E9628
:102FC000DFAE2E972F96EFAE2F976096FFAE6097ED
:102FD000B701A60189819A810E94BC0E6B017C0118
:102FE000C114D104E104F10409F0D4C0B501A40175
:102FF00029968EAD9FAD29970E94290A8C01F1E098
:103000004F1A5108610871082996AEADBFAD2997D6
:103010001D964D925D926D927C925097892B09F08E
:103020004ECE2A96EFAC2A97E3FE05C00E2D006423
:103030002A960FAF2A972996EEADFFAD299785A561
:1030400096A5A7A5B0A92796EEADFFAD2797848FCB
:10305000958FA68FB78F0B8D1C8D11A300A3B80180
:103060002996AEADBFAD29978C910E94A40E6B013D
:103070007C012796EEADFFAD2797C682D782E0860A
:10308000F186C8014C960E9427094B015C012796E6
:10309000AEADBFAD27971A968D929D92AD92BC9220
:1030A0001D972996EEADFFAD29971196FC93EE93EF
:1030B0008581968113969C938E9312972A96FFADE5
:1030C0002A971E96FC931E971F961C921F97589640
:1030D0001D921D921D921C925B97FD01108A118A10
:1030E000128A138A2A96FFAD2A97F5FFD5C081145C
:1030F0009104A104B10409F4CFC050968D929D9221
:10310000AD92BC9253972996EEADFFAD29974184BD
:103110005284612C712C99E0440C551C661C771C60
:103120009A95D1F7481459046A047B0408F07BC0CF
:10313000B701A6012796AEADBFAD27978D919C91A3
:103140000E94BC0E6B017C0184189508A608B70884
:10315000B2E0CB16D104E104F10408F4A6C0EFEF0D
:10316000CE16DE06EE06FE0609F4A2C04814590487
:103170006A047B04E8F200E010E02796EEADFFADB4
:103180002797C48AD58AE68AF78A0115110509F0BE
:1031900096CD53C0B1E0CB16D104E104F10409F49B
:1031A00099C1EFEFCE16DE06EE06FE0609F489C0E1
:1031B00000E010E098012D964FAD2D972E965FAD53
:1031C0002E972F966FAD2F9760967FAD6097C101B8
:1031D0000E94140B8C01892B09F071CDF1018189BA
:1031E0009289A389B489458956896789708D8A0136
:1031F0009B01025011092109310980179107A2078B
:10320000B30750F40196A11DB11D818B928BA38B46
:10321000B48B848181608483C416D506E606F706E4
:1032200008F4CACEE3CE2796AEADBFAD279754962D
:10323000CD92DD92ED92FC925797D501C401917029
:10324000AA27BB27892B8A2B8B2B31F1B701A6012B
:1032500029968EAD9FAD29970E943809462F572F8A
:10326000BC01411551056105710509F433C189E0BF
:10327000B694A794979487948A95D1F7840E951E57
:10328000A61EB71E2796AEADBFAD279758968D9256
:103290009D92AD92BC925B972C968EAD9FAD2C9774
:1032A000CF5ADF4FE2E10C948C3F02E010E065CF93
:1032B00001E010E062CF04E010E001CD09E010E091
:1032C00004CD01E010E0FBCC7801012B09F48AC0A9
:1032D0004F85588969897A89C70115E0880F991F38
:1032E0001A95E1F7481B590B61097109CE01019646
:1032F0000E94E8118C01892B09F0E1CCCE014D969A
:103300000E947609982EADE08A2EBCE12B2EB2E009
:103310003B2EDD24DA944F89588D698D7A8DC30157
:103320000E94290A8C01892B09F0C9CCCE2C8B8DE7
:103330009C8D62969FAF8EAF6297D3011B964D9086
:103340005C90FC0195862FE023871486128E138EE5
:10335000AE2DA150BB0B8A9E90018B9E300D112487
:10336000FFE0AF2EF2E0BF2EF5018591AF0190E0B6
:103370000F3F1F4F09F0E3CD6296AEADBFAD629730
:10338000A80FB91FDC921196DC925A010FEF1FEFC4
:103390002416350649F70F3F1F4F49F0220F331F00
:1033A000D201A20FB31F8D919C91892B11F46894C7
:1033B000C6F86296AEADBFAD6297CC9201E0F30164
:1033C000038360E070E0CE0101960E94A9108C0199
:1033D000892B09F074CC11E0E11AF108E114F10431
:1033E00009F099CF4F89588D698D7A8DC3010E945C
:1033F000290A8C01892B09F062CCEB8DFC8D80E2CF
:10340000DF011D928A95E9F7AB8DBC8D8BE0FE0143
:103410007D9601900D928A95E1F7EB8DFC8D88A544
:103420008871848781E0F30183832A96FFAD2A9710
:10343000F8602A96FFAF2A972A96EFAC2A97E3FE08
:10344000FACD0E940F39EB8DFC8D66877787808BD4
:10345000918BEB8DFC8D668B778B808F918F0B8D95
:103460001C8DB8012996AEADBFAD29978C910E94F5
:10347000A40E2B013C0180E2F8018387EB8DFC8DCB
:10348000128E138E2996AEADBFAD29978C918330E5
:1034900011F4148A158AEB8DFC8D148E158E168E00
:1034A000178E81E02996EEADFFAD299783834114F5
:1034B00051046104710409F4B4CD85A496A4A7A4B1
:1034C000B0A829803A80F1E04F16510461047104DC
:1034D00009F065CD02E010E0F2CB8C0125CDA4E02F
:1034E000B0E0E5E7FAE10C94703F7C011B018A0132
:1034F0002B833C83EB81FC8111821082BE016F5FC4
:103500007F4F0E94A8095C01892B09F05AC0F7017E
:103510008785A82EB12C811154C0868580FF10C1EB
:1035200082859385A485B58540895189628973898F
:10353000841B950BA60BB70BA80160E070E0841705
:103540009507A607B70708F48C015801A114B10428
:10355000C1F1F70180899189A289B38989809A8014
:10356000AC01BD01517066277727452B462B472BB1
:1035700009F0BFC0F4010185128501501109AC01A9
:10358000BD01E9E07695679557954795EA95D1F79E
:103590000423152301151105B9F5F701892B8A2B91
:1035A0008B2BA1F44681578160857185423051058E
:1035B00061057105B8F482E0F701878752E0A52E16
:1035C000B12CC5012496E2E10C948C3F44895589C5
:1035D00066897789808191810E94BC0E462F572F82
:1035E000BC01E4CF4F3FFFEF5F076F077F0739F460
:1035F00081E0F7018787AA24A394B12CE2CFF701D9
:10360000448B558B668B778BF70144895589668986
:103610007789C4010E9438092B013C0141145104EF
:103620006104710441F2400E511E611C711CA11411
:10363000F2E0BF0608F458C06501CD2CDD24C69425
:10364000F4018185928598012C0D3D1D8217930709
:1036500018F46C01C01AD10A8601A3019201B101CC
:10366000F40181810E941E24892B11F6F4018381CB
:103670008823E9F085A596A5A7A5B0A98419950981
:10368000A609B709A60160E070E084179507A607B0
:10369000B70768F4DC01BA2FAA27BB0FA20DB31D30
:1036A000F19680E092E001900D920197E1F7DC2C19
:1036B000CC24DD0CAC18BD08EB81FC8180819181AC
:1036C0008C0D9D1D918380832C0C3D1CF7018089FE
:1036D0009189A289B3898C0D9D1DA11DB11D808B7F
:1036E000918BA28BB38B32CFF701408E518E628EBD
:1036F000738EF701C088D188F1E0DF2280E092E08C
:103700008C199D096C01A816B90608F46501F7012A
:10371000408D518D628D738DC4010E94290A892BC1
:1037200009F066CFB4016F5C7F4FF7018089918902
:103730009170680F791FA601C1010E94A942BACFFA
:1037400087E0A82EB12C3DCFA6E0B0E0EAEAFBE18D
:103750000C94703F7C016B837C834A012D833E83F4
:10376000AD81BE811D921C92BE016F5F7F4F0E9492
:10377000A8093C01892B09F069C0F7018785682EEB
:10378000712C811163C0868581FF8AC180899189EE
:10379000A289B389AC01BD01480D591D611D711D80
:1037A000481759076A077B0718F44C0180949094D6
:1037B0008114910409F443C0F70180899189A28999
:1037C000B389A980BA80AC01BD0151706627772703
:1037D000452B462B472B09F035C1F5010185128594
:1037E00001501109AC01BD01E9E076956795579547
:1037F0004795EA95D1F7042315230115110509F022
:103800005BC0892B8A2B8B2B31F5D70116964D91F6
:103810005D916D917C911997411551056105710577
:1038200001F540E050E0BA01C7010E94780F462F31
:10383000572FBC01411551056105710591F4D70160
:103840001E968C911E9780641E968C93C3012696BB
:10385000E2E10C948C3FF7014489558966897789A8
:10386000E3CF413051056105710539F482E0F7017C
:10387000878772E0672E712CE9CF4F3FFFEF5F071C
:103880006F077F0741F481E0D7011F968C93662470
:103890006394712CDBCFF701448B558B668B778B50
:1038A00086819781A085B185892B8A2B8B2B21F46A
:1038B0004683578360877187F50145A556A567A59F
:1038C00070A9F701808D918DA28DB38D481759078E
:1038D0006A077B0729F4C5010E94D409892B99F650
:1038E000D70154964D915D916D917C915797C5018B
:1038F0000E9438091B012C01211431044104510498
:1039000009F4B4CF200E311E411C511C8114B2E0C9
:103910009B0608F477C06401CD2CDD24C694F50124
:103920008185928598012C0D3D1D8217930718F40F
:103930006C01C01AD10A8601A20191016B817C81C0
:10394000D50111968C910E947824892B09F09BCF88
:10395000F50185A596A5A7A5B0A982199309A40983
:10396000B509A60160E070E084179507A607B707C0
:10397000A8F495012F5C3F4FFC01FE2FEE27FF0FAF
:103980008B819C81E80FF91F80E092E0D9010190C2
:103990000D920197E1F7D50113961C92DC2CCC24F3
:1039A000DD0C8C189D08AD81BE818D919C91119785
:1039B0008C0D9D1D8D939C93EB81FC81EC0DFD1D69
:1039C000FC83EB83F70180899189A289B3898C0DEF
:1039D0009D1DA11DB11D808B918BA28BB38B428548
:1039E000538564857585481759076A077B0710F466
:1039F000AC01BD01D7011A964D935D936D937C93F5
:103A00001D97D6CEF70140895189628973898285D5
:103A10009385A485B585481759076A077B0768F021
:103A2000C5010E94D409892B09F02DCFD5019D969F
:103A30002D923D924D925C92D097F701208E318E5F
:103A4000428E538ED7015096CD90DC90B1E0DB22B0
:103A5000E0E0F2E0EC19FD096F018E169F0608F414
:103A60006401D70158964D915D916D917C915B9762
:103A7000C5010E94290A892B09F005CFF501F196AD
:103A8000D70150968D919C919170A6016B817C819C
:103A90008E0F9F1F0E94A94281E0F501838381CF91
:103AA00087E0682E712CD2CEA2E0B0E0EAE5FDE11D
:103AB0000C94783F6C01BE016F5F7F4F0E94A80994
:103AC0009C01892B09F0C5C0D6011E968C9186FFFA
:103AD000C0C00E940F395B018C01E980FA80F601B9
:103AE000448D558D668D778DC7010E94290A9C01F2
:103AF000892B09F0AEC0D6019096ED91FC9191977B
:103B000083858062838716968D919C911797169670
:103B10004D915D916D917C9119972D913C91938F71
:103B2000828FD9018C91833029F4AB0166277727E6
:103B3000448B558BD6011A964D915D916D917C9178
:103B40001D97448F558F668F778FA68AB78A008F0F
:103B5000118F128A138A81E0F7018383C7010E94C3
:103B6000D4099C01892B09F070C0D7018C91833056
:103B700009F05CC014968C911497813009F056C0FE
:103B800080E092E0B7016F5C7F4FFB019C011192D6
:103B900021503040E1F785E5F701E15DFD4F80837D
:103BA0008AEA3196808382E5D1968C93D197D2961A
:103BB0008C93D29781E6D3968C93D39791E4D49645
:103BC0009C9322E77B9720833196208331969083C4
:103BD00031968083F70181899289A389B489E75E50
:103BE000FD4F80839183A283B383F70185859685FA
:103BF000A785B089E35EFD4F80839183A283B38361
:103C0000F701858D968DA78DB0A19C01AD012F5F29
:103C10003F4F4F4F5F4F25A736A747A750AB01E057
:103C200010E081810E947824F701148240E050E086
:103C300060E0D70111968C910E94E7249C0191E0ED
:103C4000232B09F490E0292F30E0F60186858F7B45
:103C50008687C9012296EAE00C94943FA2E0B0E086
:103C6000E4E3FEE10C947E3F8C010E94541D9C0114
:103C7000892B61F4BE016F5F7F4FC8010E94A809C4
:103C80009C01892B19F4F80111821082C901229636
:103C9000E4E00C949A3FACE0B0E0E1E5FEE10C9486
:103CA000703F8C016A017B01BE016F5F7F4F0E94F4
:103CB000A8098B839C832B813C81232B09F01FC196
:103CC000D8011F968C911F97E82FF0E0FC83EB83BF
:103CD000811115C11A964D915D916D917C911D9741
:103CE00050968D919D910D90BC91A02D4C155D0528
:103CF0006E057F0508F068C0F801268521FF62C0C7
:103D0000108A118A128A138A29803A80F1018184EB
:103D10009284A12CB12C29E0880C991CAA1CBB1CF4
:103D20002A95D1F70097A105B10509F488C09C0137
:103D3000AD0121503109410951092D833E834F8343
:103D40005887D701C6010197A109B10989879A87C8
:103D5000AB87BC87BC01CD01A50194010E94363F11
:103D600029013A016D817E818F819885A501940199
:103D70000E94363F421653066406750608F45FC07B
:103D800088279927DC0188199909AA09BB092D817F
:103D90003E814F81588582239323A423B523F801C4
:103DA000808B918BA28BB38BC81AD90AEA0AFB0AC3
:103DB00044895589668977894115510561057105E1
:103DC00071F04EC06A017B01F801108A118A128AD3
:103DD000138AC114D104E104F10409F095CFC12C78
:103DE000D12C7601F80180899189A289B389428515
:103DF000538564857585481759076A077B0738F42A
:103E000082879387A487B58726852064268791704B
:103E1000AA27BB27892B8A2B8B2B09F470C0F801AA
:103E2000808D918DA28DB38D8C159D05AE05BF053E
:103E300009F465C0C08ED18EE28EF38E60C0D801C9
:103E400016964D915D916D917C9119974115510593
:103E500061057105F1F1F801448B558B668B778B09
:103E6000F80180899189A289B3898C149D04AE04DC
:103E7000BF0408F464C0F80180899189A289B389DC
:103E80008C0D9D1DAE1DBF1D808B918BA28BB38BA6
:103E9000D701C6019170AA27BB27892B8A2B8B2BB0
:103EA00009F49DCFC1010E943809462F572FBC014C
:103EB0004115510561057105D1F089E0F694E7944B
:103EC000D794C7948A95D1F7C40ED51EE61EF71E67
:103ED00089CF40E050E0BA01C8010E94780F462F18
:103EE000572FBC01413051056105710571F482E025
:103EF000D8011F968C93E2E0F0E0FC83EB838B818A
:103F00009C812C96E2E10C948C3F4F3FFFEF5F07C2
:103F10006F077F0739F481E0D8011F968C93E1E0A9
:103F2000F0E0EBCFD80116964D935D936D937C93A3
:103F30001997F801448B558B668B778B3DCF260103
:103F40003701481859086A087B08880D991DAA1D71
:103F5000BB1DF801808B918BA28BB38B868581FF73
:103F60000EC0C8010E94780F6B017C01C114D104FE
:103F7000E104F10451F440E050E0BA017CCF8081CB
:103F800091810E94BC0E6B017C01BFEFCB16DB065A
:103F9000EB06FB0609F4BFCFE2E0CE16D104E10444
:103FA000F10408F4A4CFF10185899689A789B08D21
:103FB000C816D906EA06FB0608F099CFD801549630
:103FC000CD92DD92ED92FC925797B701A601730155
:103FD000620146CFA4E0B0E0E0EFFFE10C947C3F4B
:103FE0008C017C836B8329E030E0892B09F445C088
:103FF00040E0BE016F5F7F4FCE0103960E940F0C21
:104000009C01892B89F4E980FA80D801ED92FC9219
:104010006B817C81C8010E94D8139C01009741F0FC
:10402000049711F425E030E0D8011D921C9225C0C0
:10403000F80187A187FD0EC0848184FFF3CF628DD4
:10404000738DD7018C910E94A40EF801668377834B
:1040500080879187D70115968D919C91F801938364
:10406000828340E050E0BA01C8010E94E8119C013F
:1040700084309105B9F2892BB9F6C9012496E6E09E
:104080000C94983FA2E0B0E0E8E4F0E20C947E3FAC
:104090008C01BE016F5F7F4F0E94A809009719F441
:1040A000F801118210822296E4E00C949A3FA8E075
:1040B000B0E0EDE5F0E20C94703F7C018B01BE01B5
:1040C0006F5F7F4F0E94A8096C01892B51F4011585
:1040D000110561F440E050E0BA01C7010E94E81107
:1040E0006C01C6012896E2E10C948C3FD7016D90DB
:1040F0007C90AA24AA94BB24BA94D70156964D91D9
:104100005D916D917C91599741155105610571053E
:1041100009F4ABC0C3010E94290A9C01892B09F054
:1041200082C0F701428C538CD2018C91882309F410
:10413000B7C11B969C911B979F739483853E09F48E
:104140007FC08E3209F47CC0292F2F71283009F4EA
:1041500077C09F3009F07AC086FF6FC01D96AC9083
:10416000B82EE894B6F8468557856089718940A7CE
:1041700051A762A773A7D2011D968C911D978A1132
:104180005FC05A968D919C915B97892B09F058C01E
:10419000F301238534854C914F7B4150550B6DE0E5
:1041A000649FC001659F900D11246FE072E0FCE1F7
:1041B0008F2EF2E09F2E41E050E0FB01A591BF0160
:1041C000A40DB52DB11D0D90BC91A02D411551052B
:1041D000D1F180349105A0F5AC01440F551F420F79
:1041E000531FFA01B183A083AD010196861697068D
:1041F00021F7D2016C9166FF0CC0452B51F0803441
:104200009105F0F4880F991F280F391FF9011182C9
:104210001082BA9460E070E0C7010E94A9109C016E
:10422000892B09F46ACFF701168A178A108E118E2E
:104230002430310509F030C118C08B1509F49BCF2B
:10424000BB24BA94E7CF119689F2FACFB11005C01A
:10425000C2010E9476098A1541F08FEF9FEFDC01C1
:10426000F70180A791A7A2A7B3A7F7010190F0815A
:10427000E02DFC83EB83D80156961C92F7018689CA
:104280009789A08DB18D892B8A2B8B2B09F4FBC0CC
:1042900080A591A5A2A5B3A58F3F9F4FAF4FBF4F5C
:1042A00009F088C0D7015A96AD90BC90D50180E046
:1042B00090E060E070E02EE2922E6F5F7F4F4D91B4
:1042C000242F30E0403209F487C02530310509F44D
:1042D00025EEAC014F5F5F4FF801E80FF91F693021
:1042E000710509F077C08C30910508F070C0918697
:1042F0000296F801E40FF51F2187DFCF81149104A6
:1043000029F4CA01985D8115984068F121014A1885
:104310005B08C401A0E0B0E0DC019927882760E0D9
:1043200070E0842B952BA62BB72B8D839E83AF83B8
:10433000B88745EB51E0BC01CD010E94DD349C0102
:104340008F3F910561F158F192E049165104E0F177
:10435000F801EA0DFB1D368B278B82E090E0A80E5A
:10436000B91E40E050E0A2E06A0E711C4A01AB8128
:10437000BC811B96ED91FC91E60DF71D40815181AA
:104380004115510509F0BACF95018114910411F03E
:1043900020E030E0200F311FF901168A83CF00970B
:1043A000A1F34114510481F0F801EA0DFB1D868B45
:1043B00081E0D4CF612C712C812C912CA12CB12CBB
:1043C00022242A94312CD3CF20E030E0DECF218785
:1043D000CA0173CF2187CA016B30710509F06DCF17
:1043E000F801E80FF91F1186F8012689211130C064
:1043F000892BF9F0399680E090E038E02191222372
:10440000E1F0422F022E000C550B2E3209F446C06B
:10441000BA01615471096A31710540F4D5011C96E5
:104420002C912323222311F0405E5F4F4487019695
:10443000E5CF8FE3868B81E090E0F801E80FF91F6C
:10444000168AF5018485811103C0D80119961C9242
:10445000F50183858F73D80118968C93C5014C960E
:104460000E942709F8016083718382839383D501B9
:1044700056968D919C9157979783868358968D91E8
:104480009C919583848360E070E0C7010E94A9102D
:104490009C01049709F425CE690123CE30E1C6CFF3
:1044A00024E030E0C0CE1CBC84B18F7584B9249860
:1044B0002B9A8091000181608093000108958EBD48
:1044C0000DB407FEFDCF8EB5089582E38093790881
:1044D0008FEF0E945F22982F8F3F21F08091790803
:1044E0008111F6CF21E030E09F3F11F020E030E075
:1044F000C90108952C9A16988FEF0E945F220895A3
:10450000CF93DF932C98169A8FEF0E945F220E9420
:104510006522EC01892B31F40E947A22CE01DF91D1
:10452000CF910895C1E0D0E0F9CFFF920F931F9390
:10453000CF93DF93C82FD42F152F062FF72E87FF89
:1045400009C040E050E0BA0187E30E949522823022
:1045500078F5CF770E947A220E948022892B69F118
:104560008C2F80640E945F228F2D0E945F22802FFB
:104570000E945F22812F0E945F228D2F0E945F2266
:10458000CC2351F087E8C83041F081E00E945F22DF
:10459000CC3029F48FEF01C085E90E945F22CAE088
:1045A0008FEF0E945F2287FF03C0C150C111F8CF77
:1045B000CDB7DEB7E5E00C94993F8FEFF9CFCF93FD
:1045C000DF93D82FC92F84E180937A088FEF0E9460
:1045D0005F228F3F39F480917A088111F7CF80E014
:1045E00090E01FC08E3FD9F7ED2FFC2F9F013E5F5B
:1045F0008FEF8EBD0DB407FEFDCF9EB590838EBDAF
:104600000DB407FEFDCF9EB591833296E217F307F6
:1046100081F78FEF0E945F228FEF0E945F2281E07F
:1046200090E0DF91CF9108951F93CF93DF93182FE0
:10463000D92FC62F0E9465229C01892B49F18C2F0E
:104640000E945F2221E030E0CD3F11F1E12FFD2FEC
:10465000CF019E5F20812EBD0DB407FEFDCF2181CD
:104660002EBD0DB407FEFDCF3296E817F90791F77E
:104670008FEF0E945F228FEF0E945F228FEF0E94D8
:104680005F228F7191E0853009F090E0292F30E0B2
:10469000C901DF91CF911F910895A4E0B0E0E3E557
:1046A000F3E20C947A3F8111C0C00E9453228091A2
:1046B000000181FF06C0809100012496E8E00C947F
:1046C000963F239A8EE180937A0880917A0881112F
:1046D000FCCF2B9883E080937A0880917A0881112F
:1046E000FCCF2C9A249A85B1806A85B984B1806AFE
:1046F00084B983E58CBD91E09DBD8CBD1AE08FEF40
:104700000E945F2211501111FACF40E050E0BA012F
:1047100080E00E949522182F813039F0109278089D
:104720000E947A220E945322C6CF84E680937A08A0
:104730004AEA51E060E070E088E00E949522813012
:1047400009F040C08E010F5F1F4F6E0185E0C80E5B
:10475000D11C78018FEF0E945F22F70181937F01C6
:10476000CE16DF06B9F78B818130C1F68C818A3A8B
:10477000A9F680917A08882349F040E050E060E093
:1047800070E489EA0E9495228111F3CF80917A0822
:10479000882321F240E050E0BA018AE30E9495228A
:1047A0008111BCCF8FEF0E945F22F80181938F01AE
:1047B000CE16DF06B9F7898186FD35C084E0809387
:1047C000780827C040E050E0BA0189EA0E949522AB
:1047D00001E0823010F402E019EA80917A0888231F
:1047E00041F040E050E0BA01812F0E9495228111F2
:1047F000F4CF80917A08882309F490CF40E052E00A
:1048000060E070E080E10E949522811187CF0093E3
:1048100078080E947A22809100018E7F80930001A7
:1048200080E58CBD48CF8CE0CACF81E046CF8111B6
:1048300003C080910001089583E00895EF92FF92F4
:104840000F931F93CF93DF937B01E42F952FA90143
:104850006E2F792FE801811147C0209709F444C0D9
:104860008091000180FD42C08091780883FD07C0DF
:1048700089E0440F551F661F771F8A95D1F7C13015
:10488000D105E1F481E10E94952281110BC0C7019D
:104890000E94DF229C0191E0232B09F090E0C92FB8
:1048A00080E0D82F0E947A2281E0CD2B09F480E0AD
:1048B00090E0CDB7DEB7E6E00C94983F82E10E942D
:1048C00095228111EFCFC7010E94DF22892B29F0A9
:1048D0008EEFF81A21972097B1F740E050E0BA0127
:1048E0008CE00E949522DECF84E0E2CF83E0E0CF2F
:1048F000A0E0B0E0EEE7F4E20C94783F5B016901E0
:104900007A01E80181115DC0209709F45AC08091B5
:10491000000180FD58C08091000182FD56C0809149
:10492000780883FD07C099E0CC0CDD1CEE1CFF1C51
:104930009A95D1F7C130D105F9F4B701A60188E104
:104940000E94952281113AC06EEFC5010E94142386
:104950009C0191E0232B09F090E0C92F80E0D82F33
:104960000E947A2281E0CD2B09F480E090E0CDB75F
:10497000DEB7EAE00C94943F8670882331F0AE01F4
:1049800060E070E087E90E949522B701A60189E105
:104990000E9495228111E4CF6CEFC5010E9414237F
:1049A000892B29F08EEFB81A21972097A9F76DEF80
:1049B00080E090E00E941423892B91F6C1E0D0E0C2
:1049C000CFCF84E0D3CF83E0D1CF82E0CFCFCF93DE
:1049D000DF93C4E0D0E0811106C0653041F40E944D
:1049E0005322C0E0D0E0CE01DF91CF9108958091B5
:1049F0000001C3E0D0E080FDF6CFC4E0D0E061115B
:104A00000AC00E948022C1E0D0E0892B21F00E94E0
:104A10007A22C0E0D0E00E947A22E5CF80917A0825
:104A2000882319F0815080937A088091790888232F
:104A300019F0815080937908809100011A9B07C07A
:104A40008460199906C08D7F8093000108958B7F43
:104A5000F8CF8360F9CF2898209A84E793E00197F4
:104A6000F1F700C0F89420989CEA9A95F1F70000BD
:104A700083B1809581707894E3EFF2E03197F1F79C
:104A800000C0189B8F5F0895F894209A882381F0C6
:104A90008FE08A95F1F720988DE98A95F1F700006B
:104AA000611101C0789482E08A95F1F700C0089501
:104AB00083E98A95F1F700C0209888E18A95F1F79B
:104AC00000C0EECFCF93DF93C82FD8E060E08C2FEB
:104AD00081700E944425C695D150D111F7CFDF9146
:104AE000CF910895CF93DF93C82FD7E060E08C2F4C
:104AF00081700E944425C695D150D111F7CF61E055
:104B00008C2F0E944425289A209A7894189902C0E4
:104B100020982898DF91CF910895F894209A8FE0FB
:104B20008A95F1F7209896E19A95F1F7000083B104
:104B3000789497E89A95F1F70000817008950F93A3
:104B40001F93CF93DF9308E010E0C0E0D1E00E9414
:104B50008D258111CD2BDD0F015011090115110596
:104B6000B1F78C2FDF91CF911F910F910895A4E0A1
:104B7000B0E0EDEBF5E20C947E3F8091340590912E
:104B80003505892B09F076C083E397E00197F1F7AB
:104B90000E942B25813009F06DC08CEC0E946225AB
:104BA0008EEB0E9462250BE718E019820E949F2578
:104BB000F80181938F019981982788E02CE89695D8
:104BC00008F492278A95D9F79983F8E004381F07EB
:104BD00069F7911153C080917B08803569F4809109
:104BE0007C08853049F4809180088F3F29F48091BA
:104BF0008208803109F442C080917B0890917C0842
:104C00009C01990F440B550B29833A834B835C839A
:104C1000CA01B9010E94D24020E030E040E85DE3E3
:104C200069837A838B839C8369817A818B819C8160
:104C30000E948741462F572FBC0140934705509350
:104C400048056093490570934A051092840881E0F5
:104C500080934B050E942B258CEC0E94622584E4F6
:104C60000E946225F89480E991E090933505809345
:104C7000340578942496E4E00C949A3F809184085B
:104C8000863018F010924B05E5CF8F5F8093840833
:104C9000E1CFEF92FF920F931F93CF93DF93062FF5
:104CA000142FC82FD0E0CC0FDD1F9E012B57374F9C
:104CB0007901F9019081CA57D74F961303C09881A3
:104CC000941791F0212F402F66E00E944A282091EE
:104CD000400530914105282B392B30934105209315
:104CE0004005F70100831883CDB7DEB7E6E00C94EA
:104CF000983FA2E0B0E0EFE7F6E20C947D3FF82E9B
:104D0000AE014E5F5F4F60E00E94DE2804E315E0D5
:104D1000F80124853585282B392B35872487AE016A
:104D20004F5F5F4F61E08F2D0E94DE28F8012485E0
:104D30003585282B392B3587248799818A812296BE
:104D4000E5E00C94993FA1E0B0E0E9EAF6E20C94CA
:104D5000803F91E0611101C090E0AE014F5F5F4F75
:104D6000692F0E94DE282091400530914105282BB3
:104D7000392B3093410520934005898190E021969D
:104D8000E2E00C949C3FE82FF0E0EE0FFF1FE957A4
:104D9000F74F2181408162E08C580E944A28E4E369
:104DA000F5E024853585282B392B35872487089510
:104DB00080E00E94C32608951F93CF93DF93C82FEE
:104DC000D62F142F0E94D826212F4D2F66E084E77E
:104DD0008C0F0E944A28E4E3F5E024853585282BD2
:104DE000392B35872487DF91CF911F910895E82FC4
:104DF000F0E0E957F74F9081442331F0962B9083F0
:104E000086950E94C326089560959623F8CFE82FD3
:104E1000F0E0E957F74F8081442319F0862B808317
:104E2000089560958623FBCFCF93C82F40E060E0C4
:104E300080E00E94492640E064E081E00E9407276C
:104E400041E062E081E00E940727C093870880E08C
:104E50000E94C32640E062E081E00E94F726CF91E5
:104E60000895CF9340E06FEF80E00E94492641E033
:104E700064E081E00E94072741E062E081E00E9457
:104E8000F72660E080E00E94A326C82F40E062E0A1
:104E900081E00E94F7268C2FCF910895CF93C82FE1
:104EA00040E068E081E00E94F7268C2F0E941427E2
:104EB000CF91089540E068E081E00E94F7260E94CB
:104EC00031270895CF93C82F41E068E081E00E9428
:104ED000F7268C2F0E941427CF91089541E068E0B7
:104EE00081E00E94F7260E9431270895CF93DF9337
:104EF000EC018991811103C0DF91CF9108950E9447
:104F00006227F7CFCF93DF93EC01FE0184912196C6
:104F1000811103C0DF91CF9108950E946227F5CFE0
:104F20006295660F660F607C860F80680E944E2730
:104F3000089581E00E944E2786E69EE00197F1F7F2
:104F40000000089582E00E944E2786E69EE00197C9
:104F5000F1F700000895CF9340E060E080E00E9408
:104F6000492640E068E081E00E94072740E062E0D7
:104F700081E00E94072740E064E081E00E94F7267C
:104F80002FEF8FE392E0215080409040E1F700C086
:104F900000008FE38093870880E00E94C326C3E06F
:104FA00041E062E082E00E94F72640E062E082E0B9
:104FB0000E94F7268FEF93E20197F1F700C00000FF
:104FC000C150C111EDCF88E30E944E2788E00E94B6
:104FD0004E2786E00E944E278CE00E944E27CF91FC
:104FE000089581E08093B800E9EBF0E08081808350
:104FF00008959AE08091BC0087FD07C091508DE331
:105000008A95F1F700C09111F5CF21E030E09923A6
:1050100011F020E030E0C901880F991F08958093B6
:10502000BB0084E88093BC000E94F9270895A0E0AB
:10503000B0E0EDE1F8E20C94793FD62F142FC82FA1
:10504000CC0F83E0C82ED12C04EA94E9B92E00934A
:10505000BC000E94F9277C018C2F0E940F28E82AAF
:10506000F92A8D2F0E940F28E82AF92A812F0E9401
:105070000F288E299F29B092BC0021E0C21AD108C6
:10508000C114D10411F0009711F7CDB7DEB7E9E0F4
:105090000C94953F8F929F92AF92BF92CF92DF92E6
:1050A000EF92FF920F931F93062FD42EC22E182F2C
:1050B000110F83E0E82EF12C94EA992E24E9822E38
:1050C0009092BC000E94F9275C01812F0E940F285A
:1050D000A82AB92A802F0E940F28A82AB92A8D2D24
:1050E0000E940F28A82AB92A8C2D0E940F288A29ED
:1050F0009B298092BC0021E0E21AF108E114F1043E
:1051000011F00097E9F61F910F91FF90EF90DF905B
:10511000CF90BF90AF909F908F900895A0E0B0E0A7
:10512000E4E9F8E20C94743FE62E8A01F82EFF0CB5
:1051300083E0C82ED12C94EA792E5A01A20EB31E18
:1051400024E9622E7092BC000E94F927EC018F2D99
:105150000E940F28C82BD92B8E2D0E940F28C82BF8
:10516000D92B48018A149B0481F46092BC00F1E0C1
:10517000CF1AD108C114D10411F0209719F7CE012C
:10518000CDB7DEB7EEE00C94903FF40181914F0172
:105190000E940F28C82BD92BE5CFCF93DF93EC01CA
:1051A00084EC611101C084E88093BC000E94F9275F
:1051B0002091BB002883DF91CF9108956F927F9259
:1051C0008F929F92AF92BF92CF92DF92EF92FF9217
:1051D000CF93DF9300D0CDB7DEB7D62EC42EB52E39
:1051E000682E660C862D81608A8383E0E82EF12C80
:1051F00094EAA92E24E9722EA092BC000E94F927FD
:105200004C01862D0E940F28882A992A8D2D0E94F4
:105210000F28882A992A8A810E940F28882A992A89
:10522000A092BC000E94F927882A992A60E0CE014A
:1052300001960E94CD28882A992A60E08C2D9B2D0A
:105240000E94CD28882999297092BC0021E0E21A99
:10525000F108E114F10411F0009771F60F900F902E
:10526000DF91CF91FF90EF90DF90CF90BF90AF9004
:105270009F908F907F906F900895A3E0B0E0E3E45B
:10528000F9E20C94723F562E5A018901482E440CC3
:10529000842D8160898383E0E82EF12C94EA692EC5
:1052A00024E9722E680121E0C21AD1086092BC0084
:1052B0000E94F9278A839B83842D0E940F282A81CC
:1052C0003B81282B392B3B832A83852D0E940F2875
:1052D0002A813B81282B392B3B832A837092BC0087
:1052E00032E03A95F1F700C06092BC000E94F927C5
:1052F0002A813B81282B392B3B832A8389810E9479
:105300000F282A813B81282B392B3B832A83812C30
:10531000912C8016910699F47092BC0081E0E81AF5
:10532000F108E114F10429F02A813B81232B09F0D3
:10533000BDCF8A819B812396E0E10C948E3F61E092
:10534000C814D90409F460E0C501880D991D0E94B4
:10535000CD282A813B81282B392B3B832A833FEFA1
:10536000831A930AD6CF4F925F926F927F928F9259
:105370009F92AF92BF92CF92DF92EF92FF92CF9324
:10538000DF9300D0CDB7DEB7562E642ED52EC22EB9
:10539000B32E482E440C842D81608A8383E0E82E4E
:1053A000F12C94EAA92E24E9722EA092BC000E944E
:1053B000F9274C01842D0E940F28882A992A852DCF
:1053C0000E940F28882A992A8A810E940F28882AF9
:1053D000992AA092BC000E94F927882A992A60E0A5
:1053E000CE0101960E94CD28882A992A60E0862D58
:1053F0009D2D0E94CD28882A992A60E08C2D9B2D16
:105400000E94CD28882999297092BC0021E0E21AD7
:10541000F108E114F10411F0009739F60F900F90A4
:10542000DF91CF91FF90EF90DF90CF90BF90AF9042
:105430009F908F907F906F905F904F900895A6E01F
:10544000B0E0E5E2FAE20C947C3F7B018E839D8321
:1054500000E010E020E030E040E251E4E982FA822E
:105460008E818B838D818C8369817A818B819C81F4
:105470000E94824187FF17C020E030E040E85FE3F0
:10548000E982FA828E818B838D818C8369817A8116
:105490008B819C810E94234087FD3DC0C8012696D8
:1054A000E6E00C94983F20E030E543EC57E4E982D5
:1054B000FA828E818B838D818C8369817A818B8145
:1054C0009C810E94824187FD10C020E030E543ECC2
:1054D00057E469817A818B819C810E9428407B01FD
:1054E0008E839D830B5F1F4FB5CF20E030E040E2FD
:1054F00051E4E982FA828E818B838D818C8369816C
:105500007A818B819C810E9428407B018E839D83C0
:105510000F5F1F4F9FCF2CEA35EC47E257E3E9823C
:10552000FA828E818B838D818C8369817A818B81D4
:105530009C810E94234087FF10C020E030E543ECAF
:1055400057E469817A818B819C810E9487417B012C
:105550008E839D83055011098FCF20E030E040E21B
:1055600051E4E982FA828E818B838D818C836981FB
:105570007A818B819C810E9487417B018E839D83F0
:105580000150110979CFA6E0B0E0E9ECFAE20C9401
:10559000803F8D839E8360E070E080E89FE32D81F3
:1055A0003E811216130684F02D813E81232BC9F50E
:1055B00069837A838B839C8369817A818B819C81C7
:1055C0002696E2E00C949C3F2D813E8125303105EA
:1055D000ACF020E030E543EC57E469837A838B83B9
:1055E0009C8369817A818B819C810E9487412D8176
:1055F0003E81255031093E832D83D1CF20E030E01C
:1056000040E251E469837A838B839C8369817A8148
:105610008B819C810E9487412D813E8121503109DF
:10562000EACF2D813E812C3F3F4FACF420E030E5A6
:1056300043EC57E469837A838B839C8369817A8105
:105640008B819C810E9428402D813E812B5F3F4FA2
:105650003E832D83A9CF20E030E040E251E469830E
:105660007A838B839C8369817A818B819C810E9460
:1056700028402D813E812F5F3F4FEACFFC01CB01B7
:10568000309711F009950895E0918B08F0918C08FE
:10569000309741F09F012F5F3F4F30938C0820934C
:1056A0008B0860830895BC018091890890918A08D5
:1056B0000E943E2B0895A9E3B0E0E1E6FBE20C94E2
:1056C000703F8BA79CA7DB015A019E012F5F3F4FC4
:1056D0003AA329A3FD016491662309F4CFC3CD0148
:1056E0000196653251F01C01062E000C770B8BA53C
:1056F0009CA50E943E2B8501B8C0FC01D490CD0131
:105700000296F0E3DF1245C01D0123E0220E311C9A
:1057100030E33BABFC01D490412C512C2AE2D21255
:1057200064C0D5018D919D9197FF06C0919581959B
:10573000910962E0462E512C9EA78DA7F101D590CC
:105740005D011F013EE2EE24EA94FF24FA94D31295
:1057500057C0F101D5904AE2D41609F449C01F019F
:10576000E12CF12C80ED8D0D8A3008F049C0AAE0C3
:10577000AE9DC001AF9D900D11248D0D911DD7FCE4
:105780009A957C01B0E3EB1AF108F101D5901F0165
:10579000E9CFFDE2DF1621F01C0120E22BABBCCFEC
:1057A0001D0133E0230E311CFC01D490F0E2FBAB71
:1057B00072E0472E512CB2CFEAE0ADA5BEA5EA9F1C
:1057C000C001EB9F900D11248D0D911DD7FC9A9572
:1057D0009C01205331093EA72DA7F101D5901F014F
:1057E00080ED8D0D8A3040F3ADCF1DA61EA6F8CFFB
:1057F000D501ED90FD90D4905D01C10102961C0190
:10580000ECE6DE1205C0689442F8F101D5901F0164
:10581000DD2009F433C3F8E7FD155CF021E62D1512
:105820006CF035E4D31609F473C048E5D41609F4D6
:1058300042C26D2D0D2C000C770B59CFEEE9ED0D0A
:10584000E731B8F70E2E000CFF0BED53FD4B0C9417
:10585000583F85010E5F1F4FD5016C91062E000C3D
:10586000770B8BA59CA50E943E2B5801D10132CF0E
:10587000F501A190B1908F01A114B10421F453E07E
:10588000A52E51E0B52EF50101900020E9F73197E2
:105890006F01CA18DB08F7FC04C0EC14FD0408F41F
:1058A0006701FBA98F2EFF0F990841FE20C0EA0C6B
:1058B000FB1CD5016C91662319F0AE14BF04E9F40A
:1058C000EDA5FEA5CE16DF0680F660E270E08BA5A2
:1058D0009CA50E943E2BBFEFCB1ADB0AF1CFB4018F
:1058E0008BA59CA50E943E2B2FEFC21AD20A8DA534
:1058F0009EA5C816D90698F3DACF9FEFA91AB90A60
:10590000062E000C770B8BA59CA50E943E2BD1CFB9
:10591000F50181919191A191B1918F018BA39CA3EC
:10592000ADA3BEA39C01AD01BC01CD010E943A42D2
:105930008111A5C1F7FE03C046E0E42EF12C20E062
:1059400030E0A9016BA17CA18DA19EA10E94234002
:105950002BE2C22E87FF0BC08BA19CA1ADA1BEA1E3
:10596000B0588BA39CA3ADA3BEA33DE2C32E8BA1D5
:105970009CA1ADA1BEA1BF778FA398A7A9A7BAA7E5
:105980002FEF3FEF4FE75FE7BC01CD010E943A42A6
:1059900081110FC02FEF3FEF4FE75FE76FA178A5B1
:1059A00089A59AA50E942340E2E2F2E018160CF4C1
:1059B00053C196E6D91235C0882799278E199F09B9
:1059C0000E94C32A20E030E040E05FE36FA378A7A5
:1059D00089A79AA76FA178A589A59AA50E94874152
:1059E0009B01AC016BA17CA18DA19EA10E94B73F40
:1059F000462F572FBC014BA35CA36DA37EA3CB0105
:105A0000BA010E941F2A4C0197FF02C0812C912CE1
:105A1000C701880D991D4D970CF01CC1612C712C8C
:105A200068C020E030E0A9016BA17CA18DA19EA1FE
:105A30000E942340812C912C882381F36BA17CA1AF
:105A40008DA19EA10E941F2A8E199F090E94C32A20
:105A500020E030E040E05FE36FA378A789A79AA732
:105A60006FA178A589A59AA50E9487412BA13CA189
:105A70004DA15EA16BA37CA38DA39EA36BA17CA172
:105A80008DA19EA10E94B73F4B015C016BA39CA21C
:105A90008DA3BEA26BA17CA18DA19EA10E941F2AF5
:105AA0003C01843691050CF0E7C0BAE1EB16F10435
:105AB0000CF0E2C08D399F4F24F49DE9692E7724C4
:105AC0007A94C3010E94C32A9B01AC018BA29CA2C1
:105AD000ADA2BEA26BA17CA18DA19EA10E94284077
:105AE000462F572FBC014BA35CA36DA37EA3812C33
:105AF000912CFDE2CE0101965C01CF1205C0C98256
:105B00005E0122E0A20EB11CAA27BB27AE19BF0975
:105B1000B9AFA8AFC4010E94C32A6FA7C72E7C01EA
:105B2000262F372FAC016BA17CA18DA19EA10E94D5
:105B300028406FA378A789A79AA76FA178A589A500
:105B40009AA50E949A406FA378A789A79AA78FA1C8
:105B500098A5092E000CAA0BBB0B8CAB9DABAEAB72
:105B6000BFABBC01CD010E94D2402FA53C2DA701A7
:105B70006FA778AB89AB9AAB6FA578A989A99AA9C9
:105B80000E9487419B01AC016BA17CA18DA19EA1CC
:105B90000E94B63F462F572FBC014BA35CA36DA3B9
:105BA0007EA3F5019FEF8916990611F4AEE2A19349
:105BB0008FA1805DDF018D935D01B1E08B1A9108AB
:105BC00028AD39AD821693060CF0A4CF36E6D31675
:105BD000B1F08BE277FE04C07194619471088DE29C
:105BE000D1828283C3016AE070E00E94223F605D3F
:105BF00063835F0145E0A40EB11C805D8483F501E1
:105C00001082FE013196DF010D900020E9F7119717
:105C10007D01EE1AFF0ABE2EAF2EFBA9CF2EFF0F7D
:105C2000DD0841FE3AC0CB2CDA2CD6016D916D0116
:105C3000611139C0EDA5FEA5EE16FF0608F015CEE0
:105C400060E270E08BA59CA50E943E2BBFEFEB1A93
:105C5000FB0AF0CFEFE1F2E0C9825E0182E0A80E1C
:105C6000B11C8491D5018C93BFEFAB1ABB0A31965E
:105C700084918111F7CFC3CFECE1F2E0EDCFE6E202
:105C8000F2E0DE0111965D01ECCFB6018BA59CA57B
:105C90000E943E2B2FEFE21AF20A8DA59EA5E81670
:105CA000F90698F3C0CF062E000C770B8BA59CA5A8
:105CB0000E943E2BBACF42FEBCC0F501819191916A
:105CC000A191B1918F0120E130E0782E692EABA334
:105CD000BFA3F8E7DF12BFC047E24CABDE0111966D
:105CE000B8ABAFA7812C912C6901E12CF12C672D69
:105CF000762D8BA19FA1A70196010E94363F762F9A
:105D0000872D962DABA1BFA1722E632E4BA35FA34F
:105D10006A3014F07CA9760F5401EFEFAE1ABE0A78
:105D2000705DEFA5F8A97193F8ABEFA78C159D05F1
:105D3000AE05BF0540F0F0E2AF16B10409F08EC029
:105D40008FE1882E912C40FE0BC0E1E0F0E0EC0FDB
:105D5000FD1FEA0DFB1D2DE22083C40102965C01AC
:105D600065019BA9E92E990FFF0841FE81C021E042
:105D700030E02C0F3D1FA20EB31ED5016E915D01C8
:105D8000062E000C770B8BA59CA50E943E2BE9A14B
:105D9000FAA1EA15FB0589F72DA53EA5C216D30683
:105DA00008F063CD60E270E08BA59CA50E943E2BBD
:105DB000FFEFCF1ADF0AF0CF42FE44C0F501819118
:105DC0009191A191B1918F0128E030E07ECF42FE08
:105DD0003CC0F50181919191A191B1918F0122E097
:105DE00030E073CF850142FE0CC0F50181919191A5
:105DF000A191B1918F01F4E6DF1679F02AE030E04D
:105E000064CF0E5F1F4F24E6D21222C0D5018D91C0
:105E10009C91092E000CAA0BBB0BB7FFEFCFB095DE
:105E2000A095909581959F4FAF4FBF4F689440F8D4
:105E3000E5CF20E130E0F501819191918F01A0E063
:105E4000B0E043CF28E030E0F6CF22E030E0F3CFFF
:105E50002AE030E0F0CF87E08CAB40CF450147CF60
:105E6000B7018BA59CA50E943E2BAFEFCA1ADA0A98
:105E7000EDA5FEA5CE16DF0698F379CFE996E2E10F
:105E80000C948C3F0F931F93CF93DF93182F092F00
:105E9000EB016991611105C0DF91CF911F910F91C5
:105EA0000895062E000C770B812F902F0E943E2B19
:105EB000F0CFBC018091890890918A080E94422FFE
:105EC00008950F931F93CF93DF93182F092FFB0192
:105ED0006591EF01611105C0DF91CF911F910F9185
:105EE0000895062E000C770B812F902F0E943E2BD9
:105EF000BE01EDCFBC018091890890918A080E9473
:105F0000612F0895A0E0B0E0E8E8FFE20C94803F44
:105F1000AE014B5F5F4FFA0161917191AF018091CA
:105F2000890890918A080E945B2BE2E00C949C3FC8
:105F3000A0E0B0E0EEE9FFE20C94803FAE01475FE5
:105F40005F4F6F8178858D819E810E945B2BE2E09F
:105F50000C949C3FA0E0B0E0E0EBFFE20C94803FAB
:105F60008D819E8190938C0880938B08AE01475F52
:105F70005F4F6F81788580E090E00E945B2BE0911D
:105F80008B08F0918C08108210928C0810928B086C
:105F9000E2E00C949C3FAAE0B0E0E1EDFFE20C945B
:105FA000763F89879A877B01DB011D921D921D92A6
:105FB0001C921397A985BA85ED91FC911197808168
:105FC000803211F18D3231F5CF0101968D939C9382
:105FD000818101E010E0C12CD12C8E3269F4A985B9
:105FE000BA85ED91FC911197CF0101968D939C9309
:105FF0008181CC24CA94DC2C8132C0F480E090E012
:106000002A96ECE00C94923F3196A985BA85ED93DF
:10601000FC93D0CF8B3239F4CF010196A985BA8594
:106020008D939C93818100E010E0D5CF19821A8274
:106030001B821C828E3251F5C114D104F9F6CC2496
:10604000CA94DD24DA94A985BA85ED91FC91119763
:10605000CF0101968D939C938181813258F700FF87
:1060600009C029813A814B815C81505829833A8348
:106070004B835C8389819A81AB81BC81F7018083EA
:106080009183A283B38381E090E0BACF90ED980F23
:106090009A3008F05DC0292F30E040E050E02D83B9
:1060A0003E834F835887C114D10431F520E030E09E
:1060B00040E251E469817A818B819C810E94874111
:1060C0004B015C016D817E818F8198850E94D24059
:1060D0009401A50169837A838B839C8369817A818A
:1060E0008B819C810E94B73F462F572FBC0149836B
:1060F0005A836B837C83A7CF560131E0A31AB10882
:10610000C6010E94C32A4B016C016D817E818F8183
:1061100098850E94D2409401A6016D837E838F836F
:1061200098876D817E818F8198850E9487419B0130
:10613000AC0169817A818B819C810E94B73F462F97
:10614000572FBC0149835A836B837C8365017BCFC6
:106150008F7D853409F052CFA985BA85ED91FC91E8
:106160001197CF01019611969C938E9391819D3248
:10617000E1F5CF0102968D939C939281026091325A
:1061800008F43CCF905320E030E06AE09A3008F009
:1061900035CF629FA001639F500D11249A01290FF2
:1061A000311DA985BA85ED91FC911197CF0101961A
:1061B0008D939C939181913210F501FF03C031952D
:1061C00021953109C9010E94C32A9B01AC01698153
:1061D0007A818B819C810E948741462F572FBC0179
:1061E00049835A836B837C833ACF9B3241F6CF013C
:1061F0000296A985BA858D939C939281C0CF9053C6
:106200009A3038F2FBCEFC012091DD083091DE0897
:10621000A22FA30FA37080E1A89FD0011124A35641
:10622000B74F80E101900D928A95E1F73F5F3530DD
:1062300018F43093DE0808952F5F23702093DD0853
:106240000895282F8091DD0830E0321307C020E147
:10625000829FC00111248356974F08958F5F8370EA
:106260003F5FF3CFA6E0B0E0E8E3F1E30C947C3FBE
:106270008C017B01DC011C968D919D910D90BC9150
:10628000A02D8B839C83AD83BE8340E0BC01CD01F8
:106290000E9484389F938F93F80183818F9382812A
:1062A0008F9381818F9380818F9387818F93868154
:1062B0008F9385818F9384818F9380EC92E09F935D
:1062C0008F9308E319E01F930F930E94AA2F63EBAB
:1062D00072E0C8010E947F42D8010D900020E9F7CA
:1062E0008D01AD01495359409E012F5F3F4F68E337
:1062F00079E0C7010E94A41B0FB6F894DEBF0FBE61
:10630000CDBF2696E6E00C94983FA2E0B0E0EBE823
:10631000F1E30C947E3F8C0167E972E088E399E039
:106320000E949542E8E3F9E001900020E9F7AF010F
:10633000495359409E012F5F3F4F68E379E0C80100
:106340000E94A41BC8010E942E1E2296E4E00C9419
:106350009A3FFC011082158216821782108689E30B
:106360009BE9AEE0B7E381879287A387B4878CEA85
:1063700095ECA7E2B8E385879687A787B08B118A4B
:10638000128A138A148A0895A2E0B0E0EAECF1E3DD
:106390000C947E3F8C018EE099E00E94A93183E24B
:1063A00099E00E94A9311092DE0810920109EDE8EF
:1063B000F8E01082118212821382148215821682F2
:1063C0001782148615861686178666EF72E088E3B4
:1063D00099E00E949542E8E3F9E001900020E9F796
:1063E000AF01495359409E012F5F3F4F68E379E069
:1063F000C8010E94A41B2296E4E00C949A3FAAE0F4
:10640000B0E0E5E0F2E30C94703F8D839E837A0167
:106410008B01AD81BE818C91811116C0CA01DB0157
:10642000ED81FE8181839283A383B48381E08083A5
:10643000E982FA820B831C8369817A818B819C813A
:106440002A96E2E10C948C3FAD81BE8111964D906D
:106450005D906D907C90149719962D913D914D9182
:106460005C911C9715966D917D918D919C911897DB
:106470000E94B73F5B016C01ED81FE812585368569
:10648000478550896983BA828B83DC8269817A81EE
:106490008B819C810E94B73F9B01AC0160E070E062
:1064A00080E89FE30E9428409501A60169837A83D2
:1064B0008B839C8369817A818B819C810E94874137
:1064C0001B014C01CB01D401ED81FE81818B928BAC
:1064D000A38BB48BA3019201E982FA820B831C8304
:1064E00069817A818B819C810E94B63F9101A401D0
:1064F00069837A838B839C8369817A818B819C8178
:106500000E948741A301920169837A838B839C83D4
:1065100069817A818B819C810E94B73F7B018C01CC
:106520009101A40160E070E080E89FE30E94B63F23
:106530009501A60169837A838B839C8369817A8123
:106540008B819C810E948741AD81BE8115966D93A0
:106550007D938D939C931897C701D801ED81FE819F
:1065600081839283A383B48363CFA7E0B0E0EBEB96
:10657000F2E30C947A3F8D839E838B01FB01208193
:10658000318142815381ED81FE81608171818281FF
:1065900093810E94B63F20E831E149ED57E46983D9
:1065A0007A838B839C8369817A818B819C810E9411
:1065B00087416B017C01F801248135814681578137
:1065C000ED81FE8164817581868197810E94B63F4D
:1065D00020E831E149ED57E469837A838B839C831A
:1065E00069817A818B819C810E9487418B018F8395
:1065F0009D839601A701C982DA82EB82FC826981C0
:106600007A818B819C810E9487416B017C0198017A
:106610004F815D8109831A83FF81FB838D818C8388
:1066200069817A818B819C810E9487419B01AC01A9
:10663000C982DA82EB82FC8269817A818B819C81BA
:106640000E94B73F69837A838B839C8369817A81B7
:106650008B819C810E94FA4169837A838B839C831E
:1066600069817A818B819C812796E8E00C94963F22
:10667000A8E1B0E0EEE3F3E30C94723F8C013B0140
:10668000DC0114968D919D910D90BC91A02D8D8B68
:106690009E8BAF8BB88FAC01BD018EE099E00E945C
:1066A000FF314B015C01D8018D919D910D90BC9102
:1066B000A02D898B9A8BAB8BBC8BAC01BD0183E287
:1066C00099E00E94FF316B017C019B01AC0169895B
:1066D0007A898B899C890E94B63FDC01CB01BF7708
:1066E000898B9A8BAB8BBC8B9401A5016D897E89BC
:1066F0008F89988D0E94B63FDC01CB01BF778D8BCF
:106700009E8BAF8BB88F22E539E44DE15AE3BC0193
:10671000CD010E948241181664F022E539E44DE172
:106720005AE369897A898B899C890E94824118166B
:1067300044F487E892E00E947A2F6896E0E10C9496
:106740008E3FA401B501D80114964D935D936D93CE
:106750007C931797A601B701F801408351836283A8
:106760007383C8010E9403318091DE08843009F0F0
:1067700068C081E00E9421315C0180E00E942131EB
:10678000B5010E94B5327B018C0183E00E9421316A
:106790004C0182E00E9421316C01B4010E94B532AB
:1067A0002B014C01B501C6010E94B5325B016C01A1
:1067B000DF928F93BF926F9383E792E09F938F93C3
:1067C0000E94822F0F900F900F900F900F900F90BC
:1067D0009201A401E98AFA8A0B8B1C8B69897A8958
:1067E0008B899C890E94234087FF0FC02A2D3B2D57
:1067F0004C2D5D2D69897A898B899C890E94234063
:1068000087FF03C08CE592E096CF82E00E942131A1
:106810008C01B8018DE898E00E94B53220E030E0AC
:1068200040E050E4698B7A8B8B8B9C8B69897A89E9
:106830008B899C890E94234087FF0FC083E392E0ED
:106840007ACF823008F479CF82500E9421318C01B6
:1068500086E592E00E947A2FDCCF8AE292E00E94E5
:106860007A2FD80114962D913D914D915C911797F7
:1068700060910209709103098091040990910509C2
:106880000E94B73F4B015C01CB01D5018093020907
:1068900090930309A0930409B0930509F80120819E
:1068A000318142815381609106097091070980917D
:1068B0000809909109090E94B73F6B017C01CB0147
:1068C000D7018093060990930709A0930809B09314
:1068D000090920910109213089F4F8018485958501
:1068E000A685B78580930A0990930B09A0930C099C
:1068F000B0930D0982E0809301091FCF2F5F209391
:106900000109233009F019CF20E030E040E450E4E1
:10691000898A9A8AAB8ABC8A69897A898B899C8997
:106920000E9428406D837E838F83988720E030E02B
:1069300040E450E4C98ADA8AEB8AFC8A69897A8958
:106940008B899C890E94284069837A838B839C83EE
:1069500080910A0990910B09A0910C09B0910D0941
:106960008D879E87AF87B88B10920109109202091C
:106970001092030910920409109205091092060959
:1069800010920709109208091092090910920A0939
:1069900010920B0910920C0910920D0980E1FE0172
:1069A0003196ADE8B8E001900D928A95E1F7B30118
:1069B000CE0101960E943231C0CE0F931F938B01FE
:1069C0009C01CA01003811052105310520F4CB01D5
:1069D0001F910F9108950115110541E0240731051C
:1069E000C0F4853B9140A9F4E2ECF6E080E090E051
:1069F0004591559160E070E04017510762077307B9
:106A000021F001968038910599F780589F4F99277A
:106A1000DFCF80E090E0DCCFFC01E038F10570F0E2
:106A2000653B714069F4EF3FF10509F048F4EE0F62
:106A3000FF1FEE53FA4F0590F491E02DCF0108951A
:106A4000E0E0F0E0FBCFA4E0B0E0E9E2F5E30C9495
:106A5000803F69837A838B839C8329813A814B8130
:106A60005C812115310541405105E8F589819A8104
:106A7000E4E1F4E08115A0E19A0710F4E0EDF4E020
:106A80006591749131976115710531F186179707FA
:106A900018F1AF014C5F5F4F32960590F491E02DF5
:106AA0002F2F3327FF27DB01AE0FBF1F8A179B074E
:106AB000D0F52930310580F4F901E652FD4B0C94F4
:106AC000583FFA01DDCFFC01E61BF70BEE0FFF1F6D
:106AD000E40FF51F859194919C0140E050E02983DB
:106AE0003A834B835C8369817A818B819C81249674
:106AF000E2E00C949C3F9C01261B370B217033274E
:106B0000821B930BE9CF4097E7CF8097E5CFC097E3
:106B1000E3CF4A97E1CF0896DFCF80559109DCCFCC
:106B200080569C41D9CF232B61F6EE0FFF1FE40F57
:106B3000F51FA6CF6EE978E087E59AE00E949542BE
:106B4000089560E978E087E59AE00E94954208950B
:106B50000E94A13561E878E087E69AE00E949542BC
:106B600008956BE778E087E59AE00E949542E0910E
:106B70004205E93070F4F0E0ED51FD4B0C94583FC4
:106B80001092670A08956FE678E087E69AE00E941F
:106B90009542089563E678E0F8CF66E578E0F5CFB2
:106BA00065E478E0F2CF64E378E0EFCF63E278E089
:106BB000ECCF64ED78E087E59AE00E94954266EEBE
:106BC00078E087E69AE00E949542089566EC78E0C6
:106BD00087E69AE00E949542089563E178E087E6AF
:106BE0009AE00E949542089562EC77E087E59AE08A
:106BF0000E949542E7E5FAE08EE3808B118A0895C2
:106C0000CF92DF92EF92FF9280914E05811111C0D9
:106C10006BE078E087E59AE00E94954263E078E0D7
:106C200087E69AE00E949542FF90EF90DF90CF9028
:106C30000895C0904B02D0904C02E0904D02F0902D
:106C40004E0220E030E0A901C701B6010E942340B6
:106C500087FF4CC0F7FAF094F7F8F09483E51F92A1
:106C60008F93FF92EF92DF92CF928BEF97E09F93FB
:106C70008F9387E59AE09F938F930E94AA2FC090ED
:106C80004702D0904802E0904902F0904A028DB746
:106C90009EB70A960FB6F8949EBF0FBE8DBF20E038
:106CA00030E0A901C701B6010E94234087FF20C040
:106CB000F7FAF094F7F8F09487E51F928F93FF921C
:106CC000EF92DF92CF9283EF97E09F938F9387E6C7
:106CD0009AE09F938F930E94AA2F8DB79EB70A9632
:106CE0000FB6F8949EBF0FBE8DBF9ECF8EE4B7CF78
:106CF00085E4E3CF80914E0581111BC069EE77E0FA
:106D000087E59AE00E94954280914C051F928F93EF
:106D100082ED97E09F938F9387E69AE09F938F93FE
:106D20000E94AA2F0F900F900F900F900F900F902E
:106D30000895809152028F93809151028F93809198
:106D400050028F9380914F028F938DED97E09F9328
:106D50008F9387E59AE09F938F930E94AA2F8DB718
:106D60009EB708960FB6F8949EBF0FBE8DBFCCCFCE
:106D700066EC78E0F19902C064ED78E087E59AE08E
:106D80000E9495426EED78E0F39902C066EE78E0DD
:106D900087E69AE00E9495420895A4E0B0E0E3ED12
:106DA000F6E30C947F3F8091430590914405A091B8
:106DB0004505B091460589839A83AB83BC8320E067
:106DC00030E040E850E4BC01CD010E948241181639
:106DD0000CF449C08091430590914405A09145056C
:106DE000B091460589839A83AB83BC832DEC3CEC40
:106DF0004CE650E4BC01CD010E9482411816ACF172
:106E00008091430590914405A0914505B0914605B8
:106E100089839A83AB83BC832AE939E949E550E445
:106E2000BC01CD010E948241181614F592E09983AD
:106E300080E40E944E27E98128E0E29FF0011124BE
:106E4000E950F74FFA83E98310E0E981FA818591EF
:106E5000FA83E9830E9462271F5F1830B1F72496F6
:106E6000E3E00C949B3F1982E3CFA1E0A983E0CF3C
:106E7000B3E0B983DDCFCF93DF93C82FE0914D0509
:106E800081E0C11101C080E0F0E0EE0FFF1FE2558C
:106E9000F74F0590F491E02D0995F89480913C0509
:106EA00090913D057894892BB1F5F89484E690E0B3
:106EB00090933D0580933C0578940E94CD3660E028
:106EC00080E00E949027E7E5FAE001900020E9F7D2
:106ED000EF01C855DA4087E59AE00E947627CF3067
:106EE000F8F080E00E94622761E080E00E94902735
:106EF000E7E6FAE001900020E9F7EF01C856DA4032
:106F000087E69AE00E947627C03139F0CF5F80E2B1
:106F10000E946227F9CFC111D0CFDF91CF910895A0
:106F2000CF5F80E20E946227DACF80934D050E94F6
:106F30003B370895843029F08BE00E9495378FEF1E
:106F4000089580E008959091780A890F87FD05C023
:106F500083302CF48093780A089582E0FBCF80E0A0
:106F6000F9CF823029F0883091F0813021F40895F2
:106F70008FEF0E94A337E091780A0E2E000CFF0BD2
:106F8000E55EF64F84910E9495378FEF089581E07A
:106F9000F0CFCF930E949006E0915005F0E0EE0F05
:106FA000FF1FE95EF64F0590F491E02D0995C82F7B
:106FB0008F3F41F0809150058C1721F00E94992756
:106FC000C0935005CF910895FC01228533858CE94B
:106FD000820F243681F05BE9520F452F4695469586
:106FE00067E00E94023F490F4F5F852F64E60E94D1
:106FF000023F481B842F94E0980F4085518586817D
:10700000141615063CF0890F67E00E94023F81E0EC
:10701000890F0895FA01E05CF64F6491860F890F9D
:107020004130510589F323703327232B69F78F5F94
:10703000EBCFA4E0B0E0EFE1F8E30C947E3F69838E
:107040007A838B839C83CE0101960E942A058C0152
:107050000E94E437F801208531852230310591F412
:10706000268137818E5B821B67E00E94023F8FE1A1
:10707000891B90E082179307D9F484819581029748
:10708000D4F414C029303105F9F4268137818E5BA0
:10709000821B67E00E94023F8FE1891B90E082170C
:1070A000930779F48481958102972CF081E004C0E4
:1070B00082179307DCF782E090E02496E4E00C94DA
:1070C0009A3F82179307DCCF2350310926303105D0
:1070D00068F7F1CF0E9419382BE297FF04C0919511
:1070E000819591092DE22093990A6AE070E00E944F
:1070F000223F605D60939A0A805D80939B0A1092A4
:107100009C0A89E99AE00895A8E0B0E0EAE8F8E38B
:107110000C947E3F69837A838B839C8341114BC09F
:10712000CE0101960E942A058C0124E031E03F93B4
:107130002F93D80111968C9111978F938C918F93E7
:1071400013968C9113978F9312968C9112978F931D
:1071500015968C9115978F9314968C9114978F9305
:1071600017968C9117978F9316968C9116978F93ED
:1071700018968D919C91199701969F938F931A96CB
:107180008D919C918459984F9F938F938EE199E0B4
:107190009F938F9389E79AE09F938F930E94AA2FE2
:1071A0000FB6F894DEBF0FBECDBF89E79AE02896F0
:1071B000E4E00C949A3F89819A81AB81BC81BC0147
:1071C000CD010E94193820E13EE0829FA001839FFB
:1071D000500D929F500D1124052E000C660B770B5D
:1071E00089819A81AB81BC81840F951FA61FB71F2F
:1071F00089839A83AB83BC83CE0101960E942A05C2
:107200008C0189819A81AB81BC818D839E83AF8300
:10721000B887BC01CD010E946A389C0188CFA8E0E4
:10722000B0E0E5E1F9E30C947E3F00915702109144
:1072300058022091590230915A020D831E832F83E8
:107240003887C901B8010E94193820E13EE0829FC9
:10725000A001839F500D929F500D1124052E000C0C
:10726000660B770B8091570290915802A0915902BA
:10727000B0915A02840F951FA61FB71F89839A8366
:10728000AB83BC83CE0101960E942A05FC01868156
:107290009781092E000CAA0BBB0BDC0199278827CC
:1072A00044815581052E000C660B770B3BE0440FA3
:1072B000551F661F771F3A95D1F7842B952BA62B68
:1072C000B72B42815381052E000C660B770B15E01E
:1072D000440F551F661F771F1A95D1F7842B952BE6
:1072E000A62BB72B40815181052E000C660B770B26
:1072F0007695679557954795842B952BA62BB72B9D
:107300004285538540555109052E000C660B770BBD
:1073100029E1440F551F661F771F2A95D1F7842B4B
:10732000952BA62BB72B408551854F5F5F4F052EC0
:10733000000C660B770B35E1440F551F661F771F56
:107340003A95D1F78C019D01042B152B262B372B59
:10735000C901B8012896E4E00C949A3F9C01F90118
:1073600080812F5F3F4F8132D0F08C32C1F7615066
:107370006111F5CFF901ADE9BAE08191882321F0DF
:107380008C3211F06F3141F4E62FF0E0E356F54F07
:1073900010828DE99AE008956F5F8D93EECF80E0C3
:1073A00090E00895CF92DF92EF92FF920F931F9398
:1073B000CF937C016B01F89484E690E090933905BB
:1073C00080933805789400E010E0A8958EB3817121
:1073D000811135C0F89480913805909139057894E1
:1073E000892B69F10E94EF07811104C00E945707A1
:1073F000C80113C00E94F807C82F0E949308011506
:10740000110569F4C43239F4F701C08381E090E0DA
:107410008C159D0510F080E090E08C01D6CFC8015E
:107420000196F701E00FF11FC083CA3089F7CF91B1
:107430001F910F91FF90EF90DF90CF90089580E023
:1074400090E0F5CF282FFB018491882329F0A22F0B
:10745000B92F31969D91981308952A2F9B2FF4CF21
:10746000282FE82FF92F80E090E0620F3AE06E13AA
:1074700001C00895219120532A3048F4389FA0017B
:10748000399F500D1124CA01820F911DF0CF80E069
:1074900090E00895A8E1B0E0E0E5FAE30C94783FCD
:1074A0008C0163E579E00E94223A811173C061E0AA
:1074B000C8010E94AE397C01009709F451C062E016
:1074C0000E94303A9E838D8362E0C70102960E943B
:1074D000303A9C838B8362E0C70104960E94303A65
:1074E0009A83898369E0C8010E94AE397C010097C4
:1074F000B9F162E00E94303A98878F8362E0C70159
:1075000002960E94303A01979A87898762E0C70104
:1075100004960E94303A8C599F4F9C878B87CE01EE
:1075200001960E94D204462F572FBC014093570268
:10753000509358026093590270935A024F3F5F4F25
:107540006F4F7F4F69F062E0C8010E94AE39FC01C5
:10755000892B19F08081813441F010924E05F39807
:107560001D8A1E8A1F8A188E0DC0F39A80915702B9
:1075700090915802A0915902B0915A028D8B9E8B26
:10758000AF8BB88F6D897E898F89988D6896EAE078
:107590000C94943F6CE479E0C8010E94223A811176
:1075A000DFCF66E0C8010E94AE39FC019C8B8B8B5B
:1075B0008081803319F410924E05D2CF82E08093FF
:1075C0004E0562E0C8010E94AE397C019C8B8B8B1A
:1075D00062E00E94303A9C0140E050E02D8B3E8BEF
:1075E0004F8B588FCA01B9010E94D04060934B0263
:1075F00070934C0280934D0290934E0232E0E30E62
:10760000F11CFC8AEB8A7E0143E1E40EF11CCE0101
:1076100001966C01BC01C7010E94CB2F20E030E035
:1076200040E752E469817A818B819C810E942840E5
:10763000F62FE72F462F572FBC0149835A836B83C0
:107640007C832F2F3E2FAC0160914B0270914C0236
:1076500080914D0290914E020E94B73F60934B0281
:1076600070934C0280934D0290934E0263E0C801E8
:107670000E94AE39FC019C8B8B8B80815601670187
:107680008E3489F080914B0290914C02A0914D0272
:10769000B0914E02B05880934B0290934C02A0934D
:1076A0004D02B0934E0264E0C8010E94AE397C01E5
:1076B0009C8B8B8B63E00E94303A9C0140E050E051
:1076C0002D8B3E8B4F8B588FCA01B9010E94D04041
:1076D00060934702709348028093490290934A0254
:1076E00033E0E30EF11CFC8AEB8AB501C6010E946F
:1076F000CB2F20E030E040E752E469817A818B8132
:107700009C810E942840F62FE72F462F572FBC015F
:1077100049835A836B837C832F2F3E2FAC0160916A
:107720004702709148028091490290914A020E945A
:10773000B73F609347027093480280934902909349
:107740004A0265E0C8010E94AE39FC019C8B8B8B1C
:107750008081853489F08091470290914802A09100
:107760004902B0914A02B058809347029093480270
:10777000A0934902B0934A0267E0C8010E94AE3963
:107780008B8B9C8B0E94544280934C0569E0C8010E
:107790000E94AE399C8B8B8BB501C6010E94CB2F0A
:1077A00089819A81AB81BC8180934F029093500272
:1077B000A0935102B09352028091570290915802C7
:1077C000A0915902B0915A028093530290935402AF
:1077D000A0935502B0935602C3CECDB7DEB72E9715
:1077E0000FB6F894DEBF0FBECDBF88E198E20FB6AA
:1077F000F894A895809360000FBE9093600014BE2B
:107800000B9A139A0F9A3E9A0E9A8FEF93E29093E7
:107810008900809388008AE08093810082E08093D1
:107820006F0081E080937C008FEA80937A000E9451
:1078300059080E94F12740E060E080E00E94DC26C9
:107840000E94AB270E949927789480917A008064E7
:1078500080937A0081B1846381B9809164008066ED
:107860008093640080E880BF83E895E090938A0865
:10787000809389088EE391E00E947A2F81E00E9434
:1078800095379BE1A92E91E0B92E2DE0822E21E0C3
:10789000922EA8958EB38171882339F183E391E00C
:1078A0000E947A2F82E00E949537F09B0CC083E003
:1078B0000E9495372FEF3FE34BE02150304040408E
:1078C000E1F700C0000013983799FECF5FEF8FEF0C
:1078D0009CE2515080409040E1F700C00000F498D5
:1078E000139A89E291E00E947A2F84E00E949537F2
:1078F000809142051F928F93BF92AF920E94822F78
:1079000010925702109258021092590210925A0285
:1079100019821A821B821C826091420510924205D4
:107920008AEF90E00E946207AFEFBFE32BE0A15027
:10793000B0402040E1F700C000000F900F900F9082
:107940000F90F099A6CF80E00E94172481FF04C019
:1079500081E0809342059DCF41E063E071E083E0E8
:1079600093E00E94D5159C01009771F03F938F938F
:107970009F928F920E94822F84E0809342050F9005
:107980000F900F900F9085CF82E08093420585E0A5
:1079900091E00E94592F85E00E94953761E082E3D3
:1079A00090E00E9462074698F79A3FEF4FEB56E04F
:1079B000315040405040E1F700C000000E94D8071D
:1079C000A89580E00E943B370E94B7250E94C937E6
:1079D00080913E0590913F0541E0892B09F440E0FC
:1079E00060E881E00E94F726F39904C083EF90E0FD
:1079F0000E947A2F64E670E08BE592E00E94D23913
:107A00008C01892BB1F48EB381718823C9F20E9455
:107A1000EC07469AF79881E00E948A078091420518
:107A2000873009F436CF61E084EF91E00E9462076D
:107A300030CF8BE592E00E944A3A6F83788789873E
:107A40009A878F819885A985BA850097A105B10588
:107A500009F4A7C0BC01CD010E94193820E13EE025
:107A6000DC010E945E3F6B877C878D879E87DC01EF
:107A7000CB012F81388549855A85820F931FA41F1A
:107A8000B51F89839A83AB83BC83CE0101960E9484
:107A90002A05FC0182E1A1E5B5E001900D928A95ED
:107AA000E1F7F89480913A0590913B057894892B01
:107AB00009F068C0F89484EF91E090933B058093BF
:107AC0003A057894809152058F93809151058F9358
:107AD000809154058F93809153058F938091560523
:107AE0008F93809155058F9380915B0590915C05F4
:107AF0008459984F9F938F938091590590915A057F
:107B000001969F938F93809158058F93809157058D
:107B10008F9381ED90E09F938F930E94822F8091AD
:107B2000430590914405A0914505B0914605BF934A
:107B3000AF939F938F9380EC90E09F938F930E94DD
:107B4000822F80914B050FB6F894DEBF0FBECDBFDC
:107B50008823E1F18091470590914805A09149055E
:107B6000B0914A05BF93AF939F938F9383EB90E0BF
:107B70009F938F930E94822F0F900F900F900F90E2
:107B80000F900F9041E060E181E00E94F72686E6C9
:107B90009EE00197F1F7000040E060E181E00E9483
:107BA000F726F19B2EC09E012B5F3F4FA8016BE58E
:107BB00072E081EE92E00E94A41B8D819E8180176D
:107BC000910749F085E08093420521CF8DE990E04F
:107BD0000E947A2FD7CF80914E05823031F46FED1D
:107BE00078E087E492E00E943833A895F29B09C0C0
:107BF00081EE92E00E94541D892B11F086E0E3CFC4
:107C0000F29880914E05823019F481E080934E0500
:107C100089819A81AB81BC81892B8A2B8B2B09F4BA
:107C2000CFCEF199CDCE209157023091580240919C
:107C3000590250915A022F83388749875A8741E069
:107C40006F81788589859A850E948438D82EC92EBF
:107C5000E82FF92F90E72DE28191811125C0CF9275
:107C6000DF9281E990E09F938F930BE512E01F93E1
:107C70000F930E94AA2F8CE6E82E81E0F82E1F9326
:107C80000F93FF92EF920E94822F42E1B80181EEA2
:107C900092E00E9410160FB6F894DEBF0FBECDBF63
:107CA000892B71F088E08FCF8B3231F08A33A1F6C7
:107CB000DF0111972C93D0CFDF0111979C93CCCF8C
:107CC0004091EB025091EC026091ED027091EE0256
:107CD00081EE92E00E944B1E892B21F79E012B5FC3
:107CE0003F4F42E050E061E071E081EE92E00E949F
:107CF000A41B892BB9F6A895CF92DF928AE890E071
:107D00009F938F931F930F930E94AA2F1F930F93FC
:107D1000FF92EF920E94822F42E16BE572E08FEDBD
:107D200098E00E9410160FB6F894DEBF0FBECDBFCC
:107D3000892B29F08FED98E00E942E1EB3CF409141
:107D4000E9085091EA086091EB087091EC088FED1A
:107D500098E00E944B1E892B69F78FED98E00E94F6
:107D6000C4318111E7CFA895CF92DF928CE790E0E4
:107D70009F938F931F930F930E94AA2F1F930F938C
:107D8000FF92EF920E94822F42E16BE572E08FEB4F
:107D900092E00E9410160FB6F894DEBF0FBECDBF62
:107DA000892B39F08FED98E00E942E1E81EE92E033
:107DB000C3CF4091C9025091CA026091CB02709129
:107DC000CC028FEB92E00E944B1E892B59F79E014B
:107DD0002B5F3F4F42E050E061E071E08FEB92E0BB
:107DE0000E94A41B892BF1F6A895F19A83E0809359
:107DF000420562E082E390E00E94620786E00E9412
:107E00009537DECD991B79E004C0991F961708F0CD
:107E1000961B881F7A95C9F780950895AA1BBB1BEE
:107E200051E107C0AA1FBB1FA617B70710F0A61B7A
:107E3000B70B881F991F5A95A9F780959095BC019B
:107E4000CD01089597FB072E16F4009407D077FD17
:107E500009D00E940E3F07FC05D03EF49095819515
:107E60009F4F0895709561957F4F0895A1E21A2E56
:107E7000AA1BBB1BFD010DC0AA1FBB1FEE1FFF1FCE
:107E8000A217B307E407F50720F0A21BB30BE40B1E
:107E9000F50B661F771F881F991F1A9469F7609565
:107EA0007095809590959B01AC01BD01CF0108951F
:107EB000EE0FFF1F0590F491E02D09940E94A73F5B
:107EC000B7FF0895821B930B08950E94A73FA59FBB
:107ED000900DB49F900DA49F800D911D11240895C5
:107EE0002F923F924F925F926F927F928F929F92CA
:107EF000AF92BF92CF92DF92EF92FF920F931F93B8
:107F0000CF93DF93CDB7DEB7CA1BDB0B0FB6F89468
:107F1000DEBF0FBECDBF09942A88398848885F84A8
:107F20006E847D848C849B84AA84B984C884DF8019
:107F3000EE80FD800C811B81AA81B981CE0FD11DFD
:107F40000FB6F894DEBF0FBECDBFED010895A29F1E
:107F5000B001B39FC001A39F700D811D1124911D1D
:107F6000B29F700D811D1124911D08955058BB279B
:107F7000AA270E94CE3F0C9448410E943A4138F013
:107F80000E94414120F039F49F3F19F426F40C94EB
:107F900037410EF4E095E7FB0C943141E92F0E9444
:107FA000594158F3BA17620773078407950720F001
:107FB00079F4A6F50C947B410EF4E0950B2EBA2FC4
:107FC000A02D0B01B90190010C01CA01A0011124DF
:107FD000FF27591B99F0593F50F4503E68F11A168B
:107FE000F040A22F232F342F4427585FF3CF46951C
:107FF00037952795A795F0405395C9F77EF41F163E
:10800000BA0B620B730B840BBAF09150A1F0FF0F07
:10801000BB1F661F771F881FC2F70EC0BA0F621FF3
:10802000731F841F48F4879577956795B795F795E3
:108030009E3F08F0B0CF9395880F08F09927EE0F78
:108040009795879508950E940D4108F481E0089561
:108050000E943C400C9448410E94414158F00E94CB
:108060003A4140F029F45F3F29F00C94314151111D
:108070000C947C410C9437410E94594168F3992338
:10808000B1F3552391F3951B550BBB27AA27621714
:108090007307840738F09F5F5F4F220F331F441F21
:1080A000AA1FA9F335D00E2E3AF0E0E832D0915055
:1080B0005040E695001CCAF72BD0FE2F29D0660F42
:1080C000771F881FBB1F261737074807AB07B0E885
:1080D00009F0BB0B802DBF01FF2793585F4F3AF08B
:1080E0009E3F510578F00C9431410C947C415F3FE8
:1080F000E4F3983ED4F3869577956795B795F79511
:108100009F5FC9F7880F911D9695879597F90895F8
:10811000E1E0660F771F881FBB1F62177307840794
:10812000BA0720F0621B730B840BBA0BEE1F88F7A3
:10813000E09508950E94A1406894B1110C947C418F
:1081400008950E94614188F09F5798F0B92F9927B0
:10815000B751B0F0E1F0660F771F881F991F1AF032
:10816000BA95C9F714C0B13091F00E947B41B1E0DB
:1081700008950C947B41672F782F8827B85F39F0DA
:10818000B93FCCF3869577956795B395D9F73EF4CB
:1081900090958095709561957F4F8F4F9F4F089573
:1081A000E89409C097FB3EF4909580957095619591
:1081B0007F4F8F4F9F4F9923A9F0F92F96E9BB2747
:1081C0009395F695879577956795B795F111F8CFC3
:1081D000FAF4BB0F11F460FF1BC06F5F7F4F8F4F2E
:1081E0009F4F16C0882311F096E911C0772321F024
:1081F0009EE8872F762F05C0662371F096E8862FBC
:1082000070E060E02AF09A95660F771F881FDAF712
:10821000880F9695879597F90895990F0008550F3F
:10822000AA0BE0E8FEEF16161706E807F907C0F0FC
:1082300012161306E407F50798F0621B730B840B04
:10824000950B39F40A2661F0232B242B252B21F4DE
:1082500008950A2609F4A140A6958FEF811D811D7E
:10826000089597F99F6780E870E060E008959FEFB8
:1082700080EC089500240A941616170618060906BD
:10828000089500240A94121613061406050608958C
:10829000092E0394000C11F4882352F0BB0F40F414
:1082A000BF2B11F460FF04C06F5F7F4F8F4F9F4F54
:1082B000089557FD9058440F551F59F05F3F71F0D6
:1082C0004795880F97FB991F61F09F3F79F087953D
:1082D0000895121613061406551FF2CF4695F1DFC6
:1082E00008C0161617061806991FF1CF8695710556
:1082F000610508940895E894BB2766277727CB018A
:1083000097F908950E940D4108F48FEF08950E9497
:108310009A410C9448410E943A4138F00E944141F0
:1083200020F0952311F00C9431410C943741112425
:108330000C947C410E94594170F3959FC1F3950FB5
:1083400050E0551F629FF001729FBB27F00DB11DD9
:10835000639FAA27F00DB11DAA1F649F6627B00D69
:10836000A11D661F829F2227B00DA11D621F739F52
:10837000B00DA11D621F839FA00D611D221F749F60
:108380003327A00D611D231F849F600D211D822FA7
:10839000762F6A2F11249F5750409AF0F1F08823CE
:1083A0004AF0EE0FFF1FBB1F661F771F881F9150FB
:1083B0005040A9F79E3F510580F00C9431410C9438
:1083C0007C415F3FE4F3983ED4F3869577956795BB
:1083D000B795F795E7959F5FC1F7FE2B880F911D25
:1083E0009695879597F9089519F416F40C943741EA
:1083F0000C943F420E946141B8F39923C9F3B6F34C
:108400009F57550B87FF0E944D420024A0E640EA8B
:10841000900180585695979528F4805C660F771FD9
:10842000881F20F026173707480730F4621B730BAC
:10843000840B202931294A2BA695179407942025CF
:1084400031254A2758F7660F771F881F20F0261717
:108450003707480730F4620B730B840B200D311D76
:10846000411DA09581F7B901842F9158880F9695E9
:10847000879508950E940D41880B990B08959F3FA1
:1084800031F0915020F4879577956795B795880FCF
:10849000911D9695879597F9089591505040660FD4
:1084A000771F881FD2F70895FC0188279927E89441
:1084B00021912032E9F3293010F02E30C8F32B320D
:1084C00041F02D3239F4689404C00E94B942820F01
:1084D000911D219120532A30C0F31EF4909581956F
:1084E0009F4F0895FB01DC0104C08D910590801918
:1084F00021F441505040C8F7881B990B0895FB01A7
:10850000DC010D900020E9F7119705900D920020F5
:10851000E1F70895FC010590061621F00020D9F737
:10852000C00108953197CF010895FB01DC0105904A
:108530000D920020E1F70895FB01DC0104C08D914C
:108540000190801921F441505040C8F7881B990BC5
:108550000895FB01DC0102C001900D924150504092
:10856000D8F70895DC0101C06D9341505040E0F709
:1085700008957AE0979F902D879F802D910D11246B
:108580000895F894FFCFE72E292CF22E882C882C02
:10859000192C192C192C192C192C192C192C192CB3
:1085A000DC2E192C192C192C382C192CF22E192CE4
:1085B000192C5B2E63357B358335853587358935B9
:1085C0008B358D359035C035C335C035C035CA358E
:0885D000CD35D035D335D63589
:0685D800010D0A005A002B
:00000001FF
